:020000040800F2
:1000000000070020F1010008212D0008D92C00086C
:10001000012D0008D92C0008F92C0008F301000874
:10002000F3010008F3010008F3010008BD3D0008DA
:10003000F3010008F3010008F3010008F3010008D0
:10004000F3010008F3010008F3010008F3010008C0
:10005000F3010008F301000829690008516900084C
:1000600079690008A1690008C9690008F30100085E
:10007000F3010008F3010008F3010008F301000890
:10008000F3010008F3010008F30100088D2C0008BB
:10009000B92C0008C92C0008F3010008F169000818
:1000A000F3010008F3010008F3010008F301000860
:1000B000D96A0008F3010008F3010008F301000801
:1000C000F3010008F3010008F3010008F301000840
:1000D000F3010008C56A0008F3010008F3010008F5
:1000E000556A0008F3010008F3010008F301000855
:1000F000F3010008F3010008F3010008F301000810
:10010000F3010008F3010008F3010008F3010008FF
:10011000F3010008F3010008F3010008F3010008EF
:10012000F3010008F3010008F3010008F3010008DF
:10013000F3010008F3010008F3010008F3010008CF
:10014000F3010008F3010008F3010008DD5E000878
:10015000F3010008F3010008F3010008F3010008AF
:10016000F3010008F3010008F3010008F30100089F
:10017000F3010008F3010008F3010008F30100088F
:10018000F3010008F3010008F3010008F30100087F
:10019000F3010008F3010008F3010008F30100086F
:1001A000F3010008F3010008F3010008F30100085F
:1001B000F3010008F3010008F3010008F30100084F
:1001C000F3010008F3010008F3010008F30100083F
:1001D000F3010008F3010008F3010008F30100082F
:1001E000651500080000000000000000000000008D
:1001F00002E000F000F8FEE772B6374880F30888A6
:10020000364880F3098836483649086040F20000D5
:10021000CCF200004EF63471CEF200010860BFF35C
:100220004F8FBFF36F8F40F20000C0F2F0004EF628
:100230008851CEF200010860BFF34F8FBFF36F8F7C
:100240004FF00000E1EE100A4EF63C71CEF20001D4
:100250000860062080F31488BFF36F8F05F006FB5B
:1002600006F0FEF94FF055301F491B4A91423CBF42
:1002700041F8040BFAE71D49184A91423CBF41F886
:10028000040BFAE71A491B4A1B4B9A423EBF51F82E
:10029000040B42F8040BF8E700201849184A914271
:1002A0003CBF41F8040BFAE705F0E4FA06F026FA41
:1002B000144C154DAC4203DA54F8041B8847F9E797
:1002C00000F042F8114C124DAC4203DA54F8041B12
:1002D0008847F9E705F0CCBA00070020002300208A
:1002E0000000000808ED00E00001002000070020E9
:1002F0002870000800230020BC230020C023002019
:10030000E4580020E0010008E4010008E4010008CE
:10031000E40100082DE9F04F2DED108AC1F80CD052
:10032000C3689D46BDEC108ABDE8F08F002383F3BF
:1003300011882846A047002004F0AAFDFEE704F03B
:1003400029FD00DFFEE70000F8B501F087F905F0B0
:1003500027FA074605F076FA0546A8BB1F4B9F42D1
:1003600032D001339F4232D01D4B27F0FF029A4218
:1003700030D1F8B200F012FF2E4642F2107400F0B5
:1003800013FF08B10024264601F088FD20B10320A8
:1003900000F07AF80024264635B1124B9F4203D074
:1003A00005F048FA00242646002005F003FA0EB1B5
:1003B00000F080F801F0AEFA00F064FF204600F093
:1003C000DFF800F077F8F9E72E460024D7E7044677
:1003D0000126D4E706464FF47A74D0E7010007B04F
:1003E000000008B0263A09B008B501F003F9A0F101
:1003F00020035842584108BD07B541F212030221BB
:1004000001A8ADF8043001F013F903B05DF804FB66
:1004100038B5302383F31188174803680BB104F013
:1004200003FE164A144800234FF47A7104F0F2FDDB
:10043000002383F31188124C236813B12368013B16
:100440002360636813B16368013B63600D4D2B78D3
:1004500033B963687BB9022001F0C6F932236360C7
:100460002B78032B07D163682BB9022001F0BCF96C
:100470004FF47A73636038BDC02300201104000874
:10048000E0240020D8230020084B187003280CD843
:10049000DFE800F008050208022001F09BB9022005
:1004A00001F08EB9024B00225A607047D823002019
:1004B000E024002010B501F0F1FC30B1294B0322FB
:1004C0001A70294B00225A6010BD284B284A1C463E
:1004D00019680131F8D004339342F9D16268254B91
:1004E0009A42F1D9244B9B6803F1006303F58033F2
:1004F0009A42E9D205F072F905F084F9002001F082
:10050000C7F80220FFF7C0FF1C4B1A6C00221A64C8
:10051000196E1A66196E596C5A64596E5A665A6E7B
:100520005A6942F080025A615A6922F080025A6187
:100530005A691A6942F000521A611A6922F000528F
:100540001A611B6972B64FF0E0233021C3F8084DE1
:10055000D4E9003281F311889D4683F3088810475F
:10056000B2E700BFD8230020E024002000000108EB
:1005700020000108FFFF000800230020003802408F
:100580002DE9F04F93B0AC4B00902022FF210AA838
:100590009D6801F069F9A94A1378A3B9A848012117
:1005A00003601170302383F3118803680BB104F0EA
:1005B0003BFDA44AA24800234FF47A7104F02AFDBF
:1005C000002383F31188009B13B19F4B009A1A609C
:1005D0009E4A009C1378032B1EBF002313709A4A77
:1005E0004FF0000A18BF5360D3465646D14601204B
:1005F00001F0F0F824B1944B1B68002B00F0158239
:10060000002000F0F7FF0390039B002B01DA00F0BD
:1006100081FE039B002BEDDB012001F0D1F8039B51
:10062000213B162BE3D801A252F823F089060008DB
:10063000B106000845070008EF050008EF050008AF
:10064000EF050008CF0700089F090008B908000857
:100650001B0900084309000869090008EF050008A4
:100660007B090008EF050008ED09000829070008CC
:10067000EF050008310A0008950600082907000860
:10068000EF0500081B0900080220FFF7ADFE002857
:1006900040F0F581009B0221BAF1000F08BF1C4613
:1006A00005A841F21233ADF8143000F0C1FF9EE707
:1006B0004FF47A7000F09EFF071EEBDB0220FFF77D
:1006C00093FE0028E6D0013F052F00F2DA81DFE833
:1006D00007F0030A0D10133605230593042105A81E
:1006E00000F0A6FF17E054480421F9E75848042118
:1006F000F6E758480421F3E74FF01C08404600F0A5
:10070000C9FF08F104080590042105A800F090FF36
:10071000B8F12C0FF2D1012000FA07F747EA0B0BD2
:100720005FFA8BFB4FF0000901F0EAF826B10BF0FD
:100730000B030B2B08BF0024FFF75EFE57E746486C
:100740000421CDE7002EA5D00BF00B030B2BA1D17C
:100750000220FFF749FE074600289BD0012000F049
:1007600097FF0220FFF790FE00261FFA86F840460A
:1007700000F09EFF044690B10021404600F0B0FF1B
:1007800001360028F1D1BA46044641F21213022183
:1007900005A8ADF814303E4600F04AFF27E70120D7
:1007A000FFF772FE2546244B9B68AB4207D92846CB
:1007B00000F070FF013040F067810435F3E7234B10
:1007C00000251D70204BBA465D603E46ACE7002E0A
:1007D0003FF460AF0BF00B030B2B7FF45BAF0220F9
:1007E000FFF752FE322000F005FFB0F10008FFF6DF
:1007F00051AF18F003077FF44DAF0F4A926808EB32
:10080000050393423FF646AFB8F5807F3FF742AF0E
:10081000124B0193B84523DD4FF47A7000F0EAFEE5
:100820000390039A002AFFF635AF019B039A03F861
:10083000012B0137EDE700BF00230020DC2400205E
:10084000C023002011040008E0240020D823002049
:1008500004230020082300200C230020DC23002098
:10086000C820FFF7C1FD074600283FF413AF1F2D36
:1008700011D8C5F1200242450AAB25F0030028BF7C
:10088000424683490192184400F0C8FF019A80480B
:10089000FF2100F0E9FF4FEAA8037D490193C8F367
:1008A0008702284600F0E8FF064600283FF46DAFB7
:1008B000019B05EB830537E70220FFF795FD002834
:1008C0003FF4E8AE00F02CFF00283FF4E3AE002731
:1008D000B846704B9B68BB4218D91F2F11D80A9B92
:1008E00001330ED027F0030312AA134453F8203C1F
:1008F00005934046042205A901F088FA0437804692
:10090000E7E7384600F0C6FE0590F2E7CDF8148020
:10091000042105A800F08CFE06E70023642104A84A
:10092000049300F07BFE00287FF4B4AE0220FFF7B2
:100930005BFD00283FF4AEAE049800F0D9FE0590B0
:10094000E6E70023642104A8049300F067FE002872
:100950007FF4A0AE0220FFF747FD00283FF49AAED7
:10096000049800F0D5FEEAE70220FFF73DFD0028DD
:100970003FF490AE00F0E4FEE1E70220FFF734FD23
:1009800000283FF487AE05A9142000F0DFFE042103
:100990000746049004A800F04BFE3946B9E7322020
:1009A00000F028FE071EFFF675AEBB077FF472AE9F
:1009B000384A926807EB090393423FF66BAE022078
:1009C000FFF712FD00283FF465AE27F003074F4400
:1009D000B9453FF4A9AE484600F05CFE04210590FD
:1009E00005A800F025FE09F10409F1E74FF47A703B
:1009F000FFF7FAFC00283FF44DAE00F091FE00280E
:100A000044D00A9B01330BD008220AA9002000F031
:100A100033FF00283AD02022FF210AA800F024FF4B
:100A2000FFF7EAFC1C4804F039FA13B0BDE8F08F78
:100A3000002E3FF42FAE0BF00B030B2B7FF42AAEEE
:100A40000023642105A8059300F0E8FD074600286F
:100A50007FF420AE0220FFF7C7FC804600283FF459
:100A600019AEFFF7C9FC41F2883004F017FA059877
:100A700000F08EFF464600F043FF3C46B7E50646D1
:100A800052E64FF0000905E6BA467EE637467CE6B8
:100A9000DC23002000230020A0860100094A1368FF
:100AA00049F2690099B21B0C00FB01331360064B3D
:100AB000186844F2506182B2000C01FB0200186019
:100AC00080B27047182300201423002010B50021A5
:100AD0001022044600F0C8FE034B03CB2060616087
:100AE0001868A06010BD00BF107AFF1FF0B5ADF50B
:100AF000517D6EAC4FF4C47207460D46204600216E
:100B000000F0B2FE02F014F9244B4FF47A72B0FBFD
:100B1000F2F0186093E80700022384E807000DF55F
:100B2000ED702382FFF7D2FF44F204731C49238443
:100B300006A806F077F8212384F832310DF2EB2273
:100B400006AB0DF1380C1E4603CE664510605160B1
:100B5000334602F10802F6D1337813700FAE3146F6
:100B60000122204600F036FF00230393AB7E029360
:100B700005F11903019380B20123CDE904600093CC
:100B8000E97E04A3D3E90023384602F0E7FC0DF523
:100B9000517DF0BD9E6AC421818A46EEE824002082
:100BA000346C00082DE9F0412C4C237ADAB08046F1
:100BB0000D465BBB27A9284601F032F807460028FE
:100BC00042D19DF89D60C82E3ED801464FF4A662E2
:100BD000204600F049FE4FF48073C4F8F8314FF41A
:100BE0000073C4F80C334FF44073C4F82034324619
:100BF0000DF19E0104F1090000F010FE26449DF85D
:100C00009C30777223720BB9EB7E23728122002114
:100C100006AC27A800F028FE0122214627A801F0F3
:100C200045F800230393AB7E029305F1190380B2CC
:100C300001932823CDE904400093E97E05A3D3E97D
:100C40000023404602F08AFC5AB0BDE8F08100BFA4
:100C5000AFF3008026417272DF25D7B73035002010
:100C6000F0B5254E4FF48A7505FB0065F1B096F896
:100C7000D83085F8DC300024D822214685F8E840B9
:100C80003AA800F0F1FD06F1090000F0E5FDD5F805
:100C9000E4308DF8F000C2B206AF06F109010DF1A3
:100CA000F100CDE93A3400F0B9FD394601223AA805
:100CB00001F032F880B2CDE9047008230127CDE9B4
:100CC000023706F1D803019330230093317A0B48A1
:100CD00007A3D3E9002302F041FCA04206DD02F0A5
:100CE00027F8C5F8E000384671B0F0BD2046FBE7B4
:100CF00078F6339F93CACD8D303500200035002023
:100D00002DE9F0411D4D1E4E1E4F86B0284602F0C3
:100D100051FC034658B30024CDE90344ADF8144018
:100D2000027B8DF8142099684068029403AA03C2DC
:100D30001B68DFF8548043F00043029301F0FAFF90
:100D4000821941F10003009402A9384601F08EFA9D
:100D5000A04205DD284602F031FC88F80040D5E7C6
:100D600098F80030072B05D8013388F8003006B01A
:100D7000BDE8F081014802F021FCF8E700350020D1
:100D800040420F00683A0020653A002070B50D46D9
:100D900014461E4602F03EFB50B9022E10D1012C23
:100DA0000ED112A3D3E90023C5E90023012007E0F7
:100DB000282C10D005D8012C09D0052C0FD00020EC
:100DC00070BD302CFBD10BA3D3E90023ECE70BA3C0
:100DD000D3E90023E8E70BA3D3E90023E4E70BA35F
:100DE000D3E90023E0E700BFAFF30080401DA1205E
:100DF00026812A0B78F6339F93CACD8D9E6AC42133
:100E0000818A46EE26417272DF25D7B7F017304A45
:100E100039059E5638B505460E4C0021013500F0C7
:100E20005FFCA4F82C55B4F82C0500F041FC78B117
:100E3000B4F82C0500F04CFC014648B9B4F82C0578
:100E400000F04EFCB4F82C350133A4F82C35EAE759
:100E500038BD00BF3035002010B50A4B0A4A1A6071
:100E600003F5805393F870203AB9DC6E2CB120461C
:100E700001F092F8204601F0CFF9BDE81040034898
:100E800001F08AB8683A0020F46C0008C04A0020DB
:100E90002DE9F04F8FB000AF05460C4602F0BAFACC
:100EA00000284BD1237E022B1BD1E38A012B18D1C2
:100EB00001F03EFF0646FFF7F1FD03464FF4C87010
:100EC000DFF8D482B3FBF0F206F5167602FB10339E
:100ED00016FA83F3C8F80030E37E33B9A74B00223B
:100EE0001A703C37BD46BDE8F08F07F1240120465B
:100EF00000F04AFE0028F4D107F11400FFF7E6FDE8
:100F000097F8264007F11401224607F1270005F063
:100F100057FE0028E2D10F2C08D8984B1C70D8F847
:100F20000030A3F51673C8F80030DAE797F82410FC
:100F30000029D6D0284602F065FAD2E7E38A282BAA
:100F400033D010D8012B2BD0052BCAD1BFF34F8F34
:100F50008B498C4BCA6802F4E0621343CB60BFF349
:100F60004F8F00BFFDE7302BBBD1874EE17E327A39
:100F70009142B6D1607E3146002291F8DC50854224
:100F800000F0AD800132042A01F58A71F5D1326892
:100F900040F6B831FA328A4294BF32603160A0E73D
:100FA00021462846FFF7A2FD9BE721462846FFF78A
:100FB000F9FD96E7B2F8EC507B6005F103094FEAC2
:100FC00099094FEA8902D11DC908A8EBC1039D46C2
:100FD000EB460021584600F047FC04F1EE012A469A
:100FE0003144584600F01AFC7B6813B9012000F028
:100FF0004FFB96F8D20000F05BFB044630B930722C
:1010000000F08EFB204600F043FBB0E0D6F8D42081
:101010003AB996F8D200B6F82C25824201D8FFF7EB
:10102000F9FED6F8D4202A44944208D296F8D20089
:10103000B6F82C250130824201D8FFF7EBFE70682C
:101040005FFA89F2594600F017FC08B9C54679E005
:10105000726896F8D2002A447260D6F8D42005EB64
:101060000209C6F8D49000F023FB814509D396F815
:10107000D220D6F8D4000132001B86F8D220C6F860
:10108000D400FF2D0FD80024347200F049FB204615
:1010900000F0FEFA00F002FF3C4B188108B9FFF7A0
:1010A00009FAC5461DE7BB6896F8D9000AFB03623A
:1010B000FB68D2F8E41082F8E83001F58061C2F8EC
:1010C000E030C2F8E410FFF7CBFDFFF719FE96F809
:1010D000D920013202F0030286F8D920B6E74FF496
:1010E0008A7A0AFB02F505F1EA013144204600F054
:1010F00047FEF86000287FF4F4AE3544012285F8FD
:10110000E82001F015FED5F8E020D6ED007ADFEDFD
:10111000206A801A192838BF192040F6B832904248
:1011200028BF1046B8EE677A07EE900AF8EEE77A25
:1011300067EEA67ADFED176AE7EE267AFCEEE77A2D
:10114000C6ED007A96F8D9307168BB600AFB03F4EB
:10115000321992F8E8505DB1D2F8E4308B42E8469B
:101160003FF428AF002182F8E810C2F8E010C5462D
:101170007368064A9B0A01331381B2E6F9340020F2
:1011800000ED00E00400FA0530350020E8240020DE
:10119000CDCCCC3D6666663FFC340020014B187018
:1011A000704700BFF424002030B54FF000542C4BA2
:1011B00022689A4285B023D1637D0BB3294A2A481D
:1011C0001370237D03724FF48073C0F8F8314FF42D
:1011D0000073C0F80C3300254FF44073C0F820347E
:1011E0002249C0F8E450C922093000F017FB20461C
:1011F000E022294600F038FB0124204605B030BD2E
:1012000004F02AFB044608B90024F6E7184A194DF1
:10121000136C43F000731364AA6D174B9A42F3D119
:101220002B6E013B7E2BEFD8144A07CA01AB83E833
:1012300007001846032100F0FFFD6B6D83424FF05D
:101240000003E1D12A6D8A4201BFAB65054B2A6ECE
:101250001A7003BF0A4BEA6D1A601C46CDE700BF47
:101260009AAD44C5F424002030350020160000203B
:1012700000380240006600405041A0B0586600406F
:101280001023002037B51A4D00F008FE02236B71C1
:10129000184B288119681848012201F0E3FB00234C
:1012A0000193164B164900931648174B4FF4805282
:1012B00002F080F8154B197811B1124802F0A2F82B
:1012C00001F036FD0446FFF7E9FB4FF4C873B0FBAD
:1012D000F3F202FB130304F5167010FA83F00C4BC3
:1012E000186004F0AFFA08B10F232B8103B030BDB2
:1012F000E824002010230020683A00208D0D00080B
:10130000F824002000350020910E0008F42400206D
:10131000FC3400202DE9F04F2DED028B0FF238291F
:10132000D9E90089834C93B00BAE9FED7E8BFFF71C
:10133000E7FC814FDFF828A200230A93ADF8343090
:101340000B9373604FF0000B5B468DED008B012516
:101350000DF11D0207A938468DF81C508DF81DB0FF
:1013600001F02EFB9DF81C30002B40F0A58020469C
:1013700002F050F80646002845D1704F01F0D8FC25
:101380003B6898423FD301F0D3FC8246FFF786FBCF
:101390004FF4C873B0FBF3F202FB13030AF51670A7
:1013A00010FA83F03860664F97F800B0CBF1100A5E
:1013B000BBF1000F14BF33462B465FFA8AFA0EA822
:1013C0008DF82830FFF782FBBAF1060F28BF4FF0E7
:1013D000060A0EAB03EB0B0152460DF1290000F09B
:1013E0001DFA0AAB0393182302930AF10102554B2D
:1013F000D2B2CDE90053049220464CA3D3E9002396
:1014000002F04EF83E7001F093FC4F4A4F4D1368C6
:10141000C31AB3F57A7F2ED3106001F08BFC02461D
:101420000B46204602F0D4F8204601F0F3FF10B33B
:101430002B7A474E002B14BF03230223737101F054
:1014400077FC0EAF4FF47A730122B0FBF3F039460C
:101450003060304600F070FB182302933D4B01933F
:1014600080B240F25513CDE90370009342464B46DB
:10147000204602F015F82B7A93B101F059FC0026B2
:1014800007464FF48A7A95F8D900304400F00300FB
:101490000AFB005393F8E82092B30136042EF2D1F0
:1014A000C82003F0FBFC2B7A002B7FF43DAF13B078
:1014B000BDEC028BBDE8F08FDAF8143083F4805372
:1014C000CAF81430594610220EA800F0CDF90DF1DB
:1014D0001E0308AA0AA9384600F0CEFF96E80300CA
:1014E0000FAB83E803009DF834308DF844300A9B3D
:1014F0000E930EA9DDE90823204602F03DFA21E70C
:10150000D3F8E02042B12B68FA2B38BFFA23BA1A7D
:101510000533B2EB430FC0D3FFF7A2FB0028BCD1C9
:10152000BEE700BF0000000000000000401DA12039
:1015300026812A0B00350020683A0020FC34002068
:10154000F9340020F8340020603A002030350020C3
:10155000E8240020643A0020F1C6A7C1D068080F33
:101560000004024008B5054801F024F8BDE8084031
:10157000034A0449002005F0FFBA00BF683A002082
:101580009C4B0020590E00082DE9F84F4FF47A7358
:10159000DFF85880DFF8589006460D4602FB03F747
:1015A000002498F900305A1C5FFA84FA01D0A34253
:1015B00012D159F8240003682A46D3F820B03146E6
:1015C0003B46D847854207D1074B012083F800A04E
:1015D000BDE8F88F0124E4E7002CFBD04FF4FA704B
:1015E00003F05CFC0020F3E7904B00201C2300205C
:1015F0002023002007B50023024601210DF107003A
:101600008DF80730FFF7C0FF20B19DF8070003B049
:101610005DF804FB4FF0FF30F9E700000A4608B51B
:101620000421FFF7B1FF80F00100C0B2404208BDC5
:1016300030B4074B0A461978064B53F8214023680B
:10164000DD69054B0146AC46204630BC604700BF13
:10165000904B002020230020A086010070B503F0ED
:101660004DFF094E094D308000242868338883429D
:1016700008D903F03DFF2B6804440133B4F5803FE3
:101680002B60F2D370BD00BF924B0020504B002066
:1016900003F0E4BF00F1006000F58030006870479F
:1016A00000F10060920000F5803003F06DBF000093
:1016B000054B1A68054B1B889B1A834202D91044BC
:1016C00003F016BF00207047504B0020924B0020C3
:1016D000024B1B68184403F013BF00BF504B00209F
:1016E000024B1B68184403F023BF00BF504B00207F
:1016F00010F003030AD1B0F5047F05D200F10050C9
:10170000A0F51040D0F80038184670470023FBE7DA
:1017100000F10050A0F51040D0F8100A704700000A
:10172000064991F8243033B10023086A81F8243047
:101730000822FFF7B5BF0120704700BF544B0020BF
:10174000014B1868704700BF002004E070B5194BCA
:101750001D68194B0138C5F30B0408442D0C0422F5
:101760001E88A6420BD15C680A46013C82421346A1
:101770000FD214F9016F4EB102F8016BF6E7013A8E
:1017800003F10803ECD181420B4602D22C2203F86C
:10179000012B0A4A05241688AE4204D1984284BF20
:1017A000967803F8016B013C02F10402F3D1581A58
:1017B00070BD00BF002004E0986C0008846C000835
:1017C000022802BF024B4FF080529A61704700BF5F
:1017D00000040240022802BF024B4FF480529A617B
:1017E000704700BF00040240022801BF024A53694B
:1017F00083F48053536170470004024070B504467F
:101800004FF47A764CB1412C254628BF412506FB82
:1018100005F003F043FB641BF4E770BD10B5002333
:10182000934203D0CC5CC4540133F9E710BD0000EF
:1018300010B5013810F9013F3BB191F900409C42CD
:1018400003D11AB10131013AF4E71AB191F900203C
:10185000981A10BD1046FCE703460246D01A12F94A
:10186000011B0029FAD1704702440346934202D07B
:1018700003F8011BFAE770472DE9F8431F4D1446A2
:1018800095F824200746884652BBDFF870909CB339
:1018900095F824302BB92022FF2148462F62FFF70C
:1018A000E3FF95F82400C0F10802A24228BF2246B7
:1018B000D6B24146920005EB8000FFF7AFFF95F8E6
:1018C0002430A41B1E44F6B2082E17449044E4B200
:1018D00085F82460DBD1FFF723FF0028D7D108E08B
:1018E0002B6A03EB82038342CFD0FFF719FF002856
:1018F000CBD10020BDE8F8830120FBE7544B00204A
:10190000024B1A78024B1A70704700BF904B0020B0
:101910001C23002038B5194C194D204602F00CFE4E
:101920002946204602F034FE2D68EA6ED2F80438CB
:1019300043F00203C2F804384FF47A70FFF75EFFF9
:101940001049284602F02CFFEA6E0F4DD2F80438F9
:1019500028680E4923F00203C2F80438A0424FF46D
:1019600061430B6001D002F047FD6868A04204D0DB
:10197000BDE83840054902F03FBD38BD8050002029
:10198000346E00083C6E0008202300207C4B0020B1
:1019900070B50C4B0C4D1E780C4B55F826209A4216
:1019A00004460DD00A4B002114221846FFF75CFFB5
:1019B0000460014655F82600BDE8704002F01CBDE9
:1019C00070BD00BF904B00202023002080500020DD
:1019D0007C4B00202DE9F3470D460446002190463C
:1019E000284640F27912FFF73FFF234620220021CC
:1019F000284601F063FF231D02222021284601F022
:101A00005DFF631D03222221284601F057FFA31D1D
:101A100003222521284601F051FF04F1080310227A
:101A20002821284601F04AFF04F11003082238213A
:101A3000284601F043FF04F1110308224021284603
:101A400001F03CFF04F1120308224821284601F06E
:101A500035FF04F1140320225021284601F02EFF07
:101A600004F1180340227021284601F027FF04F1F9
:101A700020030822B021284601F020FF04F12103B1
:101A80000822B821284601F019FF04F12207C026D8
:101A90003B46314608222846083601F00FFFB6F5CE
:101AA000A07F07F10107F3D194F832308DF80730A9
:101AB00031460DF107030822284601F0FFFE0026FB
:101AC00004F1330A9DF807304FEAC6099E4209F532
:101AD000A47720D394F83231502B28BF50238DF8AF
:101AE0000730B8F1000F08D139460DF1070307227E
:101AF000284601F0E3FE09F24F17002604F23314E2
:101B00009DF807309E4207EBC6010DD30731C80888
:101B100002B0BDE8F0870AEB0603082239462846E2
:101B200001F0CCFE0136CDE7A3190822284601F0CA
:101B3000C5FE0136E4E7000013B50446084600215F
:101B400001602346C0F803102022019001F0B6FE88
:101B50000198231D0222202101F0B0FE0198631D8F
:101B60000322222101F0AAFE0198A31D03222521B0
:101B700001F0A4FE019804F108031022282101F0CD
:101B80009DFE072002B010BDF7B5047F05460E4646
:101B90002CB1838A122B02D9012003B0F0BD00239F
:101BA000194607220096284601F04CFD731C00934D
:101BB000012200230721284601F044FDD4B9B31CBB
:101BC0000093052223460821284601F03BFD0D2401
:101BD000B378102BE0D83746B278BB1B934210D3B2
:101BE0002B7FA88A0734E408B3B9844294BF00204D
:101BF0000120D2E7AB8ADB00083BDB08B370082486
:101C0000E6E7FB1C0093214600230822284601F04A
:101C100019FD08340137DFE7201A18BF0120BCE79F
:101C2000F7B5047F05460E462CB1838ACA2B02D92C
:101C3000012003B0F0BD0023194600960822284673
:101C400001F000FD731CD4B908220093114623460D
:101C5000284601F0F7FC10247378C82BE8D801233C
:101C600072785F1C013B934210D32B7FA88A073404
:101C7000E408B3B9844294BF00200120D9E7AB8ABD
:101C8000DB00083BDB0873700824E5E7F3190093D9
:101C9000214600230822284601F0D4FC08343B46A4
:101CA000DEE7201A18BF0120C3E70000F7B50D4694
:101CB00004460021164628468122FFF7D5FD23461B
:101CC00008220021284601F0F9FD94F901206378EB
:101CD000002AB8BF7F238DF807309EB90DF10703A6
:101CE00007220821284601F0E9FD0F2700260234CB
:101CF0009DF807309E4207EBC60105D30731C8089F
:101D000003B0F0BD0827F1E7A3190822284601F027
:101D1000D5FD0136ECE70000F7B50E46054600217B
:101D200014463046CE22FFF79FFD2B462822002185
:101D3000304601F0C3FD2B7AC82B28BFC8238DF88D
:101D400007308CB90DF1070308222821304601F035
:101D5000B5FD30242F469DF807207B1B934205D309
:101D6000E01DC00803B0F0BD2824F3E707F1090324
:101D700021460822304601F0A1FD08340137EAE788
:101D8000F7B5047F05460E4634B1838AB3F5827FEA
:101D900002D9012003B0F0BD0096012310220021DA
:101DA000284601F04FFCDCB9B31C009309222346FE
:101DB0001021284601F046FC19247388B3F5807F72
:101DC000E7D837467288BB1B934210D32B7FA88A73
:101DD0000734E408B3B9844294BF00200120D9E756
:101DE000AB8ADB00103BDB0873801024E5E73B1D6A
:101DF0000093214600230822284601F023FC0834E2
:101E00000137DFE7201A18BF0120C3E730B5094DBD
:101E10000A4491420DD011F8013B5840082340F389
:101E20000004013B2C4013F0FF0384EA5000F6D17C
:101E3000EFE730BD2083B8EDF7B54FF0FF33DFF8A3
:101E400054C0DFF854E000EB81011A4688421CD0F0
:101E500050F8044B019401AF042417F8015B82EAA7
:101E600005620825DB18164605F1FF355241002EA4
:101E7000BCBF83EA0C0382EA0E0215F0FF05F1D124
:101E8000013C14F0FF04E8D1E0E7D843D14303B0AC
:101E9000F0BD00BF9336EAA9EBE1F042F7B5384A4E
:101EA000106851686B4603C36A46364936480823B2
:101EB00004F096FE0446002833D10A25334A106800
:101EC00051686B4603C36A4631492F48082304F022
:101ED00087FE0446002849D00369B3F5E02F45D8B2
:101EE000B0F8661040F2474291423FD1294A02447D
:101EF00002F15C018B4239D35C3B234900209E1ADE
:101F0000FFF784FF3246074604F164010020FFF723
:101F10007DFFA3689F4229D1E368984208BF00254E
:101F200024E00369B3F5E02F27D8418B40F2474204
:101F3000914220D1174A024402F110018B4218D37A
:101F4000103B114900209D1AFFF760FF2A46064604
:101F500004F118010020FFF759FFA3689E4202D147
:101F6000E368984201D00D25A8E70025284603B074
:101F7000F0BD1025A2E70C25A0E70B259EE700BFCA
:101F8000B86C0008DCFF060000000108C16C000806
:101F900090FF06000800FFF710B5037C044613B954
:101FA000006804F005FE204610BD00000023BFF3CA
:101FB0005B8FC360BFF35B8FBFF35B8F8360BFF347
:101FC0005B8F7047BFF35B8F0068BFF35B8F704719
:101FD00070B505460C30FFF7F5FF05F1080604461D
:101FE0003046FFF7EFFFA04206D930466D68FFF795
:101FF000E9FF2544281A70BD3046FFF7E3FF201A99
:10200000F9E7000070B50546406898B105F1080091
:10201000FFF7D8FF05F10C0604463046FFF7D2FF64
:102020008442304694BF6D680025FFF7CBFF013C2A
:102030002C44201A70BD000038B50C460546FFF749
:10204000C7FFA04210D305F10800FFF7BBFF04440F
:102050006868B4FBF0F100FB1144BFF35B8F012013
:10206000AC60BFF35B8F38BD0020FCE72DE9F04189
:10207000144607460D46FFF7C5FF844228BF0446B5
:10208000D4B1B84658F80C6B4046FFF79BFF30447C
:10209000286040467E68FFF795FF331A9C4203D8BC
:1020A0006C600120BDE8F0816B60A41B3B68AB60F5
:1020B0002044E8600220F5E72046F3E738B50C46F7
:1020C0000546FFF79FFFA04210D305F10C00FFF774
:1020D00079FF04446868B4FBF0F100FB1144BFF3DE
:1020E0005B8F0120EC60BFF35B8F38BD0020FCE705
:1020F0002DE9FF41884669460746FFF7B7FF6C4662
:1021000006B204EBC6060025B44209D06268206816
:1021100008EB0501FFF782FB636808341D44F3E711
:1021200029463846FFF7CAFF284604B0BDE8F081CB
:10213000F8B505460C300F46FFF744FF05F10806D9
:1021400004463046FFF73EFFA042304688BF6C6829
:10215000FFF738FF201A386020B130462C68FFF7AF
:1021600031FF2044F8BD000073B5144606460D4605
:10217000FFF72EFF844228BF04460190DCB101A97D
:102180003046FFF7D5FF019B33B93268C5E902330A
:10219000C5E9002401200CE09C4238BF019428606E
:1021A000019868608442F5D93368AB60241AEC600A
:1021B000022002B070BD2046FBE700002DE9FF4180
:1021C0000F466946FFF7D0FF6C4600B204EBC0052E
:1021D0000026AC4209D0D4F8048054F8081BB81982
:1021E0004246FFF71BFB4644F3E7304604B0BDE828
:1021F000F081000038B50546FFF7E0FF04460146D0
:102200002846FFF719FF204638BD0000012188420B
:1022100038BF084604F0B6BC08B104F0C9BC70472A
:1022200010B4026854681A4623465DF8044B1847F8
:102230000020704700207047704700000020704762
:102240000E20704700F5805090F8D800C0F3400091
:102250007047000000F5805090F9E00070470000E2
:1022600000F58050C0F8DC1001207047F7B50C680D
:10227000BDF8207014F0005473D10D7B082D70D878
:10228000302585F31188456AAE6876010CD4AC68B8
:10229000240108D4AC6814F0805460D184F3118810
:1022A000204603B0F0BD01240E6804F1180C002E86
:1022B000B8BFF6004FEA0C1CB4BF46F00406760522
:1022C00045F80C600E680FFA84FC16F0804F18BFBA
:1022D00005EB0C1E05EB0C1C1EBFDEF8806146F002
:1022E0000206CEF880610E7BCCF8846105EB041504
:1022F0008E68C5F88C614E68C5F88861DCF880513D
:1023000045F00105CCF8805141F2780500EB441C02
:10231000660105EB4414AC440444CCE900230D46AB
:10232000083401F10C0C55F804EB44F804EB654556
:10233000F9D12D882580841904F5805407F0030510
:1023400094F8946026F00B06354384F894500024EA
:1023500084F31188009700F035FD0120A1E70224E5
:10236000A2E74FF0FF309CE713B500F580540191D0
:10237000E06EFFF747FE1F280AD90199E06E202280
:10238000FFF7B6FEA0F120035842584102B010BD3D
:102390000020FBE708B5302383F3118800F5805057
:1023A000C06EFFF703FE002383F3118808BD000011
:1023B00000220260828142608260704710B5002274
:1023C0000023C0E900230023044603810C30FFF7FB
:1023D000EFFF204610BD0000F0B5054600F5805027
:1023E0000C4690F8D83013F0040FC3F3800108BFF7
:1023F000114661F3820380F8D83005EB441303F5EE
:102400008453103389B01B79D8074FEA44162FD56F
:1024100082B319072ED46846FFF7D0FF05EB4413AB
:1024200003F5845303AA03F1080718685968144692
:1024300003C40833BB422246F7D1186820609B884A
:10244000A380DDE90E23CDE900230123ADF8083098
:102450002B6869461B6C28469847354405F584551A
:1024600010352B791A075CBF43F008032B7101E08C
:10247000002AF2D109B0F0BD2DE9F0479A4688B0A4
:10248000074688469146302383F3118807F5805428
:102490006846FFF793FFE06EFFF79AFD1F282AD9E1
:1024A000E06E20226946FFF7A5FE202823D103AD68
:1024B000444605AB2E4603CE9E4220606160354601
:1024C00004F10804F6D130682060B388A380DDE908
:1024D0000023C9E90023BDF80830AAF80030002322
:1024E00083F3118853464A464146384608B0BDE852
:1024F000F04700F02BBC002080F3118808B0BDE845
:10250000F08700002DE9F84F182204460F460430EA
:102510000021FFF7A9F92046234B40F8283BFFF79D
:1025200047FF04F13800FFF749FF04F1580804F5AC
:1025300082554646183530462036FFF73FFFAE42FB
:10254000F9D104F580554FF480534FF00009C5E9E7
:102550001739C5F858800123EE6604F5875804F54D
:102560008456C5F8649085F8683085F87030183660
:1025700008F118084FF0000A4FF0000B46E908ABCD
:10258000A6F11800FFF714FF203646F8289C4645B0
:10259000F4D185F8E07017B1044800F0C3FB044B98
:1025A00063622046BDE8F88FF46C0008CC6C00082C
:1025B0000064004010B5044B197804464A1C1A7098
:1025C000FFF7A0FF204610BD984B00202DE9F047F3
:1025D000002950D0294B2A4FB7FBF1F599428CBF07
:1025E0000A231123581EB5FBF3FC03FB1C53C4B292
:1025F0002BB102280346F5D80020BDE8F0870CF186
:10260000FF36B6F5806FF7D2C4EBC40E0EF10303AC
:102610004FEAE309C3F3C703A4EB030809F1010A76
:102620004FF47A755FFA88F009FB05555AFA88F875
:10263000B5FBF8F5B5F5617FC1BF0EF1FF33C3F30C
:10264000C703E01AC0B25C1C50FA84F40CFB04F41B
:10265000B7FBF4F4A142CFD1013BDBB20F2BCBD8B7
:102660000138C0B20728C7D80021107116809170B8
:10267000D3700120C1E70846BFE700BF3F420F000B
:1026800040787D0170B505460E464FF47A746B6A4A
:102690005B6803F00103B34207D04FF47A7002F095
:1026A000FDFB013CF3D1204670BD0120FCE700009A
:1026B00070B5426A936913F0700F17D000230C4D68
:1026C000936141F2900400EB4312224411794E07CA
:1026D00009D5890707D5416A55F823608E601179BD
:1026E00041F0040111710133032BECD170BD00BF27
:1026F000E06C000873B51D46436A16469A68D20717
:10270000044609D59A6801219960C2F34002CDE9D7
:1027100000650021FFF760FE636A9A68D1050BD55A
:102720009A684FF480719960C2F34022CDE9006548
:1027300001212046FFF750FE636A9A68D2030BD549
:102740009A684FF480319960C2F34042CDE9006548
:1027500002212046FFF740FE04F58053D3F8DC0049
:1027600010B103681B699847204602B0BDE870406D
:10277000FFF79EBFF8B50446466A002977D106F1F7
:102780000C073868800775D006EB01153868D5F856
:10279000B00110F0040FD5F8B0011ABFC00840F026
:1027A0000040400DA062D5F8B0C11CF0020F1CBF64
:1027B00040F08040A062D5F8B40106EB011100F0B2
:1027C0000F0084F83400D1F8B80184F82C00D1F857
:1027D000B801000A84F82D00D1F8B801000C84F883
:1027E0002E00D1F8B801000E84F82F00D1F8BC01FA
:1027F00084F83000D1F8BC01000A84F83100D1F827
:10280000BC01000C84F83200D1F8BC11090E84F828
:1028100033103821396004F1440004F1280104F137
:10282000340551F8046B40F8046BA942F9D10988CA
:102830000180C4E90E2321460023A4F8403051F85A
:10284000383B20461B6C984704F5805393F8D820FA
:10285000D3F8DC0042F0040283F8D82010B10368FA
:102860001B6998472046BDE8F840FFF721BF06F1F5
:10287000100786E7F8BD000010B5044600F05AFACC
:1028800002460B4652EA030102D0013A63F100030B
:102890000449086820B12146BDE81040FFF76ABF2F
:1028A00010BD00BF944B0020F0B5302181F311889A
:1028B000DFF848E000F583511831002441F2900C14
:1028C00000EB441565442E7977070ED4F6060CD537
:1028D000D1E9007697429E4107D2466A5EF824709D
:1028E000B7602E7946F004062E710134032C01F1F5
:1028F0002001E5D1002383F31188F0BDE06C0008CE
:1029000008B5302383F31188FFF7D2FE002383F349
:10291000118808BD2DE9F041436A0446986800F02B
:10292000E050B0F1E05F0E4622D0F8B1302383F3DF
:102930001188002504F5845741F2900804EB4513F3
:1029400043441B791A0706D50135032D07F12007EB
:10295000F4D1012007E05B07F6D43946304600F099
:1029600083FA0028F0D1002383F31188BDE8F081B9
:102970000120FBE708B5302383F3118800F5805070
:10298000C06EFFF725FB002383F3118843090CBFBA
:102990000120002008BD0000F8B51D46002313707B
:1029A0000F4606461446FFF7E5FF80F00100387039
:1029B00025B129463046FFF7ADFF2070F8BD000075
:1029C0002DE9B8410C4615461F46804600F0B2F985
:1029D0000B462178024609B9287850B14046FFF7E6
:1029E00063FFFFF78DFF3B462A462146FFF7D4FFE2
:1029F0000120BDE8B881000070B5302686F311884B
:102A0000174B1A6C42F000721A641A6A42F0007294
:102A10001A621A6A22F000721A62002383F3118884
:102A200000F5805494F8D83013F0010516D1A9B1FF
:102A300086F311880321132001F012FB03211420D7
:102A400001F00EFB0321152001F00AFB94F8D830A9
:102A500043F0010384F8D83085F3118870BD00BFBE
:102A6000003802402DE9F04700F5805588B095F810
:102A7000E030012B04468846164600F28280824FE1
:102A800057F823200AB947F82300D7F800A0C4F864
:102A90001C8084F82060BAF1000F64D095F8E03013
:102AA000012B70D001212046FFF7A6FF302383F3CE
:102AB0001188626A136823F002031360626A136864
:102AC00043F001031360636A00275F6187F3118895
:102AD00001212046FFF7D6FD002800F09580E86E22
:102AE000FFF764FA04F58359BA4609F11809202260
:102AF00000216846FEF7B8FE02A8FFF759FCCDF8A2
:102B000018A06A4609EB07030DF1180E9446BCE8BD
:102B10000300F44518605960624603F10803F5D1DB
:102B2000DCF80000186020379CF804201A71602F30
:102B3000DDD195F8D8306FF38203002785F8D830BF
:102B40006A4641462046ADF80070ADF802708DF837
:102B50000470FFF73BFD636A48BB4FF400421A6004
:102B600008B0BDE8F08741F2E800FFF74FFB81466F
:102B700010B15146FFF7C6FCC7F80090B9F1000F3D
:102B80008CD10020ECE7386803681B6B984701463E
:102B9000002887D13868FFF72FFF3868036832466E
:102BA0005B684146984700287FF47CAFE9E76122E3
:102BB0001A609DF802309DF803201B06120402F4EF
:102BC000702203F040731343BDF80020C2F30902E2
:102BD00013439DF804201205022E02F4E0020CBFFC
:102BE0004FF0004100211343626A0B43D361636AD3
:102BF00013225A61626A136823F001031360394695
:102C00002046FFF73FFD08B9636AA6E795F8E03074
:102C100093BB616AD1F8002242F00102C1F80022A0
:102C2000616AD1F8002222F47C5222F00E02C1F82F
:102C30000022616AD1F8002242F46062C1F80022E9
:102C4000626AC2F81432626AC2F80432626A41F6F9
:102C5000FF71C2F80C12626AC2F84032626AC2F8AE
:102C60004432636A0122C3F81C22626AD2F800323D
:102C700023F00103C2F8003295F8D83043F0020384
:102C800085F8D8306CE700BF944B002008B500F001
:102C900051F850EA0103024602D0421E61F10001E0
:102CA000044B186810B10B46FFF724FDBDE808403F
:102CB00001F0B8B8944B002008B50020FFF7DCFD08
:102CC000BDE8084001F0AEB808B50120FFF7D4FD1B
:102CD000BDE8084001F0A6B800B59BB0EFF309814C
:102CE00068226846FEF79AFDEFF30583014B9B6B64
:102CF000FEE700BF00ED00E008B5FFF7EDFF0000C4
:102D000000B59BB0EFF3098168226846FEF786FDA7
:102D1000EFF30583014B5B6BFEE700BF00ED00E0C6
:102D2000FEE700000FB408B5029802F05DF8FEE778
:102D300002F0D4BC02F0B6BC0139C9B202299EBF70
:102D400000EBC1000023C0E901337047F8B51B88D0
:102D50005B0705460E4615D4044600F11807BC4231
:102D600010D0636853B12B682846DB6B9847A36883
:102D7000C1B23246606898470834F0E7A368002B78
:102D8000F1D1F9E70120F8BD73B56C4684E806007F
:102D9000014600224E68D5B26EB98E685EB900EB6E
:102DA000C200021D94E80300013582E803001D7093
:102DB000012002B070BD0132032A01F10801E9D1FE
:102DC0000020F6E72DE9F04F89B00446BDF84870C1
:102DD0000E46054600F118084FF0000907F00407F9
:102DE0004FF0000A4FF0000BA84538D06B680BB9C4
:102DF000AB684BB157B923682046DB6B9847AB688B
:102E0000C1B23246686898470835EDE7B9F1000F5E
:102E1000FAD1CDE900ABADF80890334603AA06F12C
:102E2000080E186859689446ACE8030008337345E7
:102E30006246F6D11868CCF800009B88ACF80430E4
:102E4000FFF778FF0423ADF808302368CDE90001CF
:102E50001B6C6946204698474FF00109D4E70120D2
:102E600009B0BDE8F08F000030B503680968DD0FD8
:102E7000B5EBD17F23F0604421F060424FEAD1707E
:102E80000BD0002BB8BFA40C0029B8BF920C944201
:102E900002D034BF0120002030BD944205D1C1F3DF
:102EA0008070C3F380738342F6D194422CBF00201C
:102EB0000120F1E72DE9F041456A15B94162BDE80D
:102EC000F0814B6823F06047C3F38A464FEAD37E14
:102ED000C3F3807816EA230638BF3E46AC462B463D
:102EE0005A68BEEBD27F22F060440AD0002A18DA7A
:102EF000A40CB44217D19D420FD10D60DEE71346FA
:102F0000EEE7A74207D102F08044C2F38072424547
:102F10000BD054B1EFE708D2EDE7CCF800100B600E
:102F2000CDE7B44201D0B442E5D81A689C46002AE5
:102F3000E5D11960C3E700002DE9F047089D01F0D5
:102F400007044FEAD508224405F0070500EBD1003D
:102F50004FF47F49944201D1BDE8F08704F00707A0
:102F600005F0070A57453E4638BF5646C6F10806E3
:102F7000111B8E4228BF0E46E10808EBD50E415CBE
:102F800013F80EC0B94029FA06F721FA0AF1FFB288
:102F90008CEA010147FA0AF739408CEA010C03F880
:102FA0000EC034443544D5E780EA0120082341F2BD
:102FB000210201B24000002980B203F1FF33B8BF03
:102FC000504013F0FF03F4D17047000038B50C46B1
:102FD0008D18A54200D138BD14F8011BFFF7E4FF9E
:102FE000F7E7000042684AB113684360438981896A
:102FF00001339BB29942438138BF838110467047A9
:1030000070B588B0202204460D4668460021FEF7C0
:103010002BFC20460495FFF7E5FF024658B16B46AE
:10302000054608AE1C4603CCB442286069602346BE
:1030300005F10805F6D1104608B070BD082817D96B
:1030400009280CD00A280CD00B280CD00C280CD046
:103050000D280CD00E2814BF4020302070470C20C3
:1030600070471020704714207047182070472020A8
:1030700070470000082817D90C280CD910280CD943
:1030800014280CD918280CD920280CD930288CBF2A
:103090000F200E207047092070470A2070470B2030
:1030A00070470C2070470D20704700002DE9F84351
:1030B000078C072F04461ED9D0E9029800254FF649
:1030C000FF73C5F12006A5F1200029FA05F108FAE1
:1030D00006F628FA00F031430143C9B21846FFF75B
:1030E00063FF0835402D0346EBD1E1693A46BDE860
:1030F000F843FFF76BBF4FF6FF70BDE8F8830000A1
:1031000010B54B6823B9CA8A63F30902CA8210BD9D
:1031100004691A681C600361C38A013BC3824A6068
:10312000EFE700002DE9F84F1D46CB8A0F46C3F3A9
:1031300009010529814692460B4630D00020AAB2EB
:1031400007F11A049EB2042E1FFA80F80FD890459A
:1031500003F1010306D3FB8A0A4462F30903FB82ED
:1031600001201AE01AF80060E6540130EAE79045C1
:10317000F1D2A1F1050B1C237C68BBFBF3F203FB2E
:1031800012BB1FFA8BF6002C45D14846FFF72AFFE9
:10319000044638B978606FF00200BDE8F88F4FF050
:1031A0000008E6E7002606607860ADB24FF0000B3D
:1031B000454510D90AEB0803221D13F8011B915550
:1031C000B1B208F101081B291FFA88F82BD0454538
:1031D00006F10106F1D8FB8AC3F30902154465F331
:1031E0000903BCE7013292B21C462368002BF9D1D7
:1031F0006B1F0B441C21B3FBF1F301339BB29A42CA
:10320000D3D2BBF1000FD0D14846FFF7EBFE20B977
:10321000C4F800B0BFE70122E7E7C0F800B05E469F
:1032200020600446C1E74545D5D94846FFF7DAFE98
:1032300008B92060AFE7C0F800B00026206004465F
:10324000B6E700002DE9F04F2DED028B1C4683B050
:103250005B69019207468846002B00F0A780238C0B
:103260002BB1E269002A00F0A180072B35D807F1C5
:103270000C00FFF7B7FE054638B96FF00205284687
:1032800003B0BDEC028BBDE8F08F14220021FEF7E5
:10329000EBFA228CE16905F10800FEF7BFFA208CF9
:1032A000013080B2FFF7E6FEFFF7C8FE013880B2BA
:1032B0002084013028746369228C1B782A4403F02F
:1032C0001F0363F03F0348F0004113723846696002
:1032D0002946FFF7EFFD0125D1E702339BB2072214
:1032E000C18A0633B3FBF2F3828A521A9BB292B2BE
:1032F0009342C2D800F10C034FF0000908EE103AD7
:103300004FF0800A4E464D4618EE100AFFF76AFE4F
:1033100083460028B1D014220021FEF7A5FA002E22
:103320003AD1019BABF8083002220BF1080E1FFACC
:1033300082FC0CF10100BCF1060F218C80B201D897
:103340008E422BD3FFF796FEFFF778FE6269127864
:10335000013802F01F028E4208BF4FF0400A42EAD5
:1033600049121BFA80F14AEA020A013048F0004291
:1033700081F808A08BF81000CBF804205946384695
:10338000FFF798FD238C0135B3422DB289F0010976
:103390004FF0000AB8D172E70022C6E7E169895D03
:1033A0000EF802100136B6B20132C0E76FF0010527
:1033B00065E70000F8B515460E46302200210446A8
:1033C0001F46FEF751FA069B6360B5F5001F079B89
:1033D000A76034BF6A094FF6FF72A36297B2E66135
:1033E00004F1100000239A4206D800230360A7824C
:1033F000E3822383E360F8BD066001333046203664
:10340000F1E7000003781BB94BB2002BC8BF017075
:103410007047000000787047F8B50C46C969074648
:1034200011B9238C002B37D1257E1F2D34D8387845
:1034300028BB228C072A2CD8268A36F003032BD1EE
:103440004FF6FF70FFF7C2FD20F00100310240048B
:1034500041EA0561400C41EA40254FF6FF722346E0
:1034600029463846FFF7EEFE002807DD626913782B
:103470000133DBB21F2B88BF00231370F8BD218AF4
:103480002D0645EA012505432046FFF70FFE0246BB
:10349000E5E76FF00300F1E76FF00100EEE70000F1
:1034A00070B58AB0044616460021282268461D469B
:1034B000FEF7DAF9BDF83830ADF810300F9B059300
:1034C0009DF840308DF81830119B07936946BDF880
:1034D0004830ADF820302046CDE90265FFF79CFF6B
:1034E0000AB070BD2DE9F041D36905460C46164679
:1034F0000BB9138C5BBB377E1F2F28D895F8008043
:10350000B8F1000F26D03046FFF7D0FD3378210206
:1035100041EAC33141EA0801338A41EA076141EADD
:1035200003410246334641F080012846FFF78AFEF8
:1035300000280ADD3378012B07D172691378013333
:10354000DBB21F2B88BF00231370BDE8F0816FF042
:103550000100FAE76FF00300F7E70000F0B58BB069
:1035600004460D4617460021282268461E46FEF7EF
:103570007BF99DF84C305A1E534253418DF8003070
:103580009DF84030ADF81030119B05939DF8483000
:103590008DF81830149B07936A46BDF85430ADF887
:1035A000203029462046CDE90276FFF79BFF0BB07D
:1035B000F0BD0000406A00B104307047436A1A68E9
:1035C000426202691A600361C38A013BC382704789
:1035D0002DE9F041D0F82080194E14461D46414691
:1035E000002709B9BDE8F081D1E90223A21A65EBF1
:1035F0000303964277EB03031ED2036A8B420DD17D
:10360000FFF77EFD036A1B68036203690B60C38AD0
:103610000161016A013BC3828846E2E7FFF770FD62
:103620000B68C8F8003003690B60C38A0161013B75
:10363000C382D8F80010D4E788460968D1E700BFF4
:1036400080841E002DE9F04F8BB00D46DDF85090C0
:1036500014469B468046002800F01981B9F1000FFE
:1036600000F01581531E3F2B00F21181012A03D176
:10367000BBF1000F40F00B810023CDE90833B8F80F
:103680001430B5EBC30F4FEAC30703D300200BB0D0
:10369000BDE8F08F2B199F42D8F80C303ABF7F1B42
:1036A000FFB227461BB9D8F81030002B7AD0272D4F
:1036B0004ED8C5F12806B7424FF000032CBFF6B232
:1036C0003E4600932946D8F8080008AB3246FFF77B
:1036D00033FCA7EB060A35445FFA8AFAB8F81430CF
:1036E00003F10053053BDB000493D8F80C3003933F
:1036F0002821039B13B1BAF1000F2CD1D8F8100088
:1037000040B1BAF1000F05D0009608AB5246691AD5
:10371000FFF712FC38B2002FB8D066070AD00AAB08
:1037200003EBD401624211F8083C02F00702134196
:1037300001F8083C082C3CD9102C40F2B580202C14
:1037400040F2B780BBF1000F00F09C80082334E00A
:10375000BA460026C2E7049BE02B28BFE02306936D
:103760000B44AB42059314D95A1B0398009692451B
:1037700034BF5246D2B2691A08AB04300792FFF741
:10378000DBFB079A1644AAEB020A1544F6B25FFA6D
:103790008AFA049B069A05999B1A0493039B1B685B
:1037A0000393A6E70093D8F8080008AB3A462946E9
:1037B000AEE7BBF1000F13D00123B4EBC30F6CD005
:1037C000082C12D89DF82030621E23FA02F2D50789
:1037D00006D54FF0FF3202FA04F423438DF820306F
:1037E0009DF8203089F8003051E7102C12D8BDF830
:1037F0002030621E23FA02F2D10706D54FF0FF32C5
:1038000002FA04F42343ADF82030BDF82030A9F8C3
:1038100000303CE7202C0FD80899631E21FA03F3EF
:10382000DA0705D54FF0FF3202FA04F40C4308948E
:10383000089BC9F800302AE7402C2BD0DDE9086549
:10384000611EC4F12102A4F1210326FA01F105FA57
:1038500002F225FA03F311431943CB0712D50122D3
:10386000A4F12003C4F1200102FA03F322FA01F1CA
:10387000A240524243EA010363EB430332432B432A
:10388000CDE90823DDE90823C9E90023FFE66FF04D
:103890000100FCE66FF00800F9E6082CA0D9102C16
:1038A000B3D9202CEED8C3E7BBF1000FADD0022373
:1038B00083E7BBF1000FBBD004237EE730B5012ABC
:1038C000144638BF0124402C85B028BF4024002571
:1038D000012ACDE9025518D81B788DF80830630706
:1038E0000AD004AB03EBD405624215F8083C02F0A1
:1038F0000702934005F8083C009103462246002148
:1039000002A8FFF719FB05B030BD082AE4D9102A38
:1039100003D81B88ADF80830E1E7202A8DBFD3E932
:1039200000231B680293CDE90223D8E710B5CB68CA
:103930001BB98B600B618B8210BD04691A681C6017
:103940000361C38A013BC382CA60F0E703064CBF30
:10395000C0F3C0300220704708B50246FFF7F6FFFB
:10396000022806D15306C2F30F2001D100F0030054
:1039700008BDC2F30740FBE72DE9F04F93B0CDE956
:1039800003230A6804461046FFF7E0FF022814BF2D
:10399000C2F306260026002A0D46824680F2F781F1
:1039A00012F0C04940F0F381097B002900F0EF815B
:1039B000022803D02378B34240F0EC81C2F30463C1
:1039C0000693104602F07F030593FFF7C5FF059BA2
:1039D00029444FEA834848EA0A4848EA4668CE78CC
:1039E00000230022CDE90823F309834648EA0008B2
:1039F000029367D0059B009302466768534608A967
:103A00002046B847002800F0C881276A4FB94146D0
:103A100004F10C00FFF7F4FA074690B96FF00200CA
:103A200054E03B6998450DD03F68002FF9D14146DD
:103A300004F10C00FFF7E4FA07460028EED0236AF1
:103A40003B60276297F817C006F01F08CCF3840C80
:103A5000ACEB08001FFA80FE0028B8BF0EF1200072
:103A6000A8EB0C031FFA83FED7E90221B8BF00B20E
:103A7000002B0793BEBF0EF120031BB2079352EA3F
:103A8000010338D0039BDFF824E39A1A049B4FF01C
:103A9000000C63EB010196457CEB01032BD36B7BA0
:103AA00097F81AE0734519D1029B002B78D00128B2
:103AB00021DC7868F8B9DFF8F0C2944570EB0103B7
:103AC00016D337E0276A27B96FF00C0013B0BDE8B2
:103AD000F08F3B699845B5D03F68F4E7B248904213
:103AE0007CEB010301D30020F0E7029B002BFAD00E
:103AF000079B0F2B17DCFA7DB30002F0030203F0E3
:103B00007C031343FB7539462046FFF7F9FA6B7BBC
:103B1000BB76029B3BB9FB7DC3F38402013262F3A7
:103B20008603FB75D0E76A7BBB7E9A42DBD1029BA2
:103B3000002B35D0B309022B32D0039BBB60049B12
:103B4000FB60142200210DA8FDF78EFE039B0A9353
:103B5000049B0B932B1D0C932B7BADF83EB0013BCC
:103B6000DBB2ADF83C30069B8DF84230059B8DF8FA
:103B7000433094F82C308DF840A083F001038DF889
:103B800044308DF84180A3680AA920469847FB7D00
:103B9000C3F38403013303F01F039B02FB82A2E7FC
:103BA000FB7DC6F34012B2EBD31F40F0F980C3F3A4
:103BB0008403434540F0FC80029A2B7BB609002A1F
:103BC00052D016F0010661D1032B40F2F480039B22
:103BD000BB60049BFB60FB8A66F30903FB822B7BC3
:103BE000AE1D033BDBB23246394604F10C00FFF751
:103BF00099FA00280CDA39462046FFF781FAFB7D56
:103C0000C3F38403013303F01F039B02FB8205E728
:103C1000DDE90884AB883B834FF6FF73C9F12000D0
:103C2000A9F1200228FA09F104FA00F0014324FA6C
:103C300002F211431846C9B2FFF7B6F909F10809B3
:103C4000B9F1400F0346E9D1B8822A7B033AD2B2D8
:103C50003146FFF7BBF9FB7DB882DA43C2F3C012ED
:103C600062F3C713FB753EE786B92E1D013BDBB23D
:103C70003246394604F10C00FFF754FA0028BADB4B
:103C80002A7BB88A013AD2B23146E2E7F98AC1F317
:103C90000901013B0429DAB25BD8281D002307F192
:103CA0001B069A4208D910F801CB06F801C0013171
:103CB00001330529DBB2F4D103990A9104990B91E0
:103CC000934207F11B010C9138BF043379680D91C1
:103CD00034BF55FA83F300230E93FB8AADF83EB050
:103CE000C3F309031A44069B8DF84230059B8DF8F7
:103CF000433094F82C30ADF83C2083F001038DF86C
:103D0000443000238DF840A08DF841807B602A7BF1
:103D1000B88A013A291DFFF759F93B8BB8828342D3
:103D200003D1A3680AA92046984720460AA9FFF7AD
:103D3000FDFDFB7DBA8AC3F38403013303F01F0347
:103D40009B02FB823B8B9A420CBF00206FF010005D
:103D5000BCE67B68002BAFD0052001E01C30334669
:103D60001E68002EFAD1091A081D2E1D184401EBF9
:103D7000090CBCF11B0F5FFA89F39DD89A429BD9BD
:103D800016F8013B00F8013B09F10109EFE76FF07C
:103D900009009BE66FF00A0098E66FF00B0095E6CD
:103DA0006FF00D0092E600BF40420F0080841E00BD
:103DB0006FF00E008AE66FF00F0087E6EFF30983DD
:103DC00005494A6B22F001024A63683383F309888C
:103DD000002383F31188704700EF00E0302080F368
:103DE000118862B60C4B0D4AD96821F4E0610904D0
:103DF000090C0A43DA60D3F8FC20094942F08072CA
:103E0000C3F8FC200A6842F001020A602022DA7737
:103E100083F82200704700BF00ED00E00003FA05C0
:103E2000001000E010B5302383F311880E4B5B685F
:103E300013F4006314D0F1EE103AEFF30984683CF8
:103E40004FF08073E361094BDB6B236684F30988D1
:103E500000F094FF10B1064BA36110BD054BFBE7CA
:103E600083F31188F9E700BF00ED00E000EF00E008
:103E70003F030008420300080268436811430160E1
:103E800003B1184770470000024AD36843F0C003EB
:103E9000D36070470010014010B5054C054A002161
:103EA000204600F087FA044A044BC4E9972310BD6A
:103EB000A04B0020893E00080010014080F0FA026B
:103EC000234A037C002918BF0A46012B30B5C0F8ED
:103ED00068220CD11F4B984209D11F4B596C41F0FD
:103EE00010015964596E41F0100159665B6EB2F9C8
:103EF00004501468D0F86032D0F85C12002D03EB47
:103F00005403B3FBF4F3BEBF23F0070503F007032C
:103F100043EA450394888B60D38843F040030B61E8
:103F2000138943F001034B6144F4045343F02C0321
:103F3000CB6004F4A05400230B60B4F5806F0B68D1
:103F40004B680CBF7F23FF2380F8643230BD00BF75
:103F5000386D0008A04B0020003802402DE9F041E8
:103F6000D0F85C62F7683368DA0504469DB20DD577
:103F7000302383F311884FF480610430FFF77CFF16
:103F80006FF480733360002383F31188302383F34D
:103F9000118804F1040815F02F033AD183F3118836
:103FA000380615D5290613D5302383F3118804F17B
:103FB000380000F07BF900284EDA0821201DFFF7B9
:103FC0005BFF4FF67F733B40F360002383F3118860
:103FD0007A0616D56B0614D5302383F31188D4E9FD
:103FE00013239A420AD1236C43B127F040073F04C0
:103FF0001021201D3F0CFFF73FFFF760002383F3E4
:104000001188D4F86822D36843B3BDE8F041106941
:1040100018472B0714D015F0080F0CBF00214FF4E0
:104020008071E80748BF41F02001AA0748BF41F06E
:1040300040016B0748BF41F080014046FFF71CFF7D
:10404000AD06736805D594F864122046194000F057
:10405000E1F93568ADB29EE77060B6E7BDE8F08182
:1040600000F1604303F561430901C9B283F800130D
:10407000012200F01F039A4043099B0003F16043B3
:1040800003F56143C3F880211A607047F8B51546FF
:1040900082680669AA420B46816938BF8568761A2C
:1040A000B54204460BD218462A46FDF7B7FBA36972
:1040B0002B44A361A3685B1BA3602846F8BD0CD901
:1040C00018463246FDF7AAFBAF1BE1683A4630447A
:1040D000FDF7A4FBE3683B44EBE718462A46FDF7EF
:1040E0009DFBE368E5E7000083689342F7B515465A
:1040F000044638BF8568D0E90460361AB5420BD251
:104100002A46FDF78BFB63692B446361A36828464D
:104110005B1BA36003B0F0BD0DD932460191FDF7E2
:104120007DFB0199E068AF1B3A463144FDF776FB11
:10413000E3683B44E9E72A46FDF770FBE368E4E700
:1041400010B50A440024C361029B8460C0E90000EA
:10415000C0E90511C1600261036210BD08B5D0E974
:104160000532934201D1826882B98268013282604D
:104170005A1C42611970D0E904329A4224BFC368C4
:104180004361002100F0A6FE002008BD4FF0FF3083
:10419000FBE7000070B5302304460E4683F3118818
:1041A000A568A5B1A368A269013BA360531CA361E4
:1041B00015782269934224BFE368A361E3690BB1D8
:1041C00020469847002383F31188284607E03146AC
:1041D000204600F06FFE0028E2DA85F3118870BDFA
:1041E0002DE9F74F04460E4617469846D0F81C9026
:1041F0004FF0300A8AF311884FF0000B154665B175
:104200002A4631462046FFF741FF034660B9414642
:10421000204600F04FFE0028F1D0002383F31188E0
:10422000781B03B0BDE8F08FB9F1000F03D0019007
:104230002046C847019B8BF31188ED1A1E448AF370
:104240001188DCE7C0E90511C160C3611144009B1E
:104250008260C0E90000016103627047F8B504465E
:104260000D461646302383F31188A768A7B1A368CB
:10427000013BA36063695A1C62611D70D4E904327A
:104280009A4224BFE3686361E3690BB12046984713
:10429000002080F3118807E03146204600F00AFE36
:1042A0000028E2DA87F31188F8BD0000D0E9052381
:1042B0009A4210B501D182687AB98268013282606F
:1042C0005A1C82611C7803699A4224BFC3688361C7
:1042D000002100F0FFFD204610BD4FF0FF30FBE74E
:1042E0002DE9F74F04460E4617469846D0F81C9025
:1042F0004FF0300A8AF311884FF0000B154665B174
:104300002A4631462046FFF7EFFE034660B9414694
:10431000204600F0CFFD0028F1D0002383F3118860
:10432000781B03B0BDE8F08FB9F1000F03D0019006
:104330002046C847019B8BF31188ED1A1E448AF36F
:104340001188DCE7026843681143016003B1184734
:10435000704700001430FFF743BF00004FF0FF33F9
:104360001430FFF73DBF00003830FFF7B9BF000041
:104370004FF0FF333830FFF7B3BF00001430FFF7C2
:1043800009BF00004FF0FF311430FFF703BF0000FA
:104390003830FFF763BF00004FF0FF323830FFF7CF
:1043A0005DBF0000012914BF6FF0130000207047AB
:1043B000FFF772BD37B515460E4A02600022426013
:1043C000C0E902220122044602740B46009000F16B
:1043D0005C014FF480721430FFF7B2FE00942B465C
:1043E0004FF4807204F5AE7104F13800FFF72AFF34
:1043F00003B030BD4C6D000810B53023044683F384
:104400001188FFF75DFD02232374002080F31188DB
:1044100010BD000038B5C36904460D461BB9042120
:104420000844FFF78FFF294604F11400FFF796FEBA
:10443000002806DA201D4FF40061BDE83840FFF780
:1044400081BF38BD026843681143016003B118475A
:104450007047000013B5446BD4F894341A6811788F
:10446000042915D1217C022912D11979128901233D
:104470008B4013420CD101A904F14C0001F0ACFFB8
:10448000D4F89444019B21790246206800F0D6F9C3
:1044900002B010BD143001F02FBF00004FF0FF3309
:1044A000143001F029BF00004C3002F001B80000C8
:1044B0004FF0FF334C3001F0FBBF0000143001F02F
:1044C000FDBE00004FF0FF31143001F0F7BE0000D8
:1044D0004C3001F0CDBF00004FF0FF324C3001F006
:1044E000C7BF00000020704710B5D0F894341A6898
:1044F00011780429044617D1017C022914D1597975
:10450000528901238B4013420ED1143001F090FEEA
:10451000024648B1D4F894444FF48073617920681E
:10452000BDE8104000F078B910BD0000406BFFF707
:10453000DBBF0000704700007FB5124B0360002313
:104540004360C0E90233012502260F4B057404467F
:104550000290019300F18402294600964FF4807383
:10456000143001F041FE094B0294CDE9006304F5DB
:1045700023724FF48073294604F14C0001F008FFC8
:1045800004B070BD746D00082D4500085544000846
:104590000B68302282F311880A7903EB82021062E1
:1045A0004A790D3243F822008A7912B103EB820373
:1045B00018620223C0F894140374002080F3118859
:1045C0007047000038B5037F044613B190F85430AB
:1045D000ABB9201D01250221FFF734FF04F11400BF
:1045E00025776FF0010100F081FC84F8545004F14C
:1045F0004C006FF00101BDE8384000F077BC38BDD9
:1046000010B5012104460430FFF71CFF0023237777
:1046100084F8543010BD000038B50446002514302D
:1046200001F0FAFD04F14C00257701F0C9FE201DD0
:1046300084F854500121FFF705FF2046BDE83840BB
:10464000FFF752BF90F85C3003F06003202B07D1D6
:1046500090F85D20212A4FF0000303D81F2A06D8C6
:1046600000207047222AFBD1C0E9143303E0034A3B
:1046700002650722426583650120704728230020D8
:1046800037B5D0F894341A681178042904461AD141
:10469000017C022917D11979128901238B40134219
:1046A00011D100F14C05284601F04AFF58B101A98B
:1046B000284601F091FED4F89444019B21790246EA
:1046C000206800F0BBF803B030BD0000F0B500EB8F
:1046D000810385B01E6A04460D46FEB1302383F384
:1046E000118804EB8507301D0821FFF7ABFEFB683E
:1046F0005B691B6806F14C001BB1019001F07AFE6A
:10470000019803A901F068FE024648B1039B2946BF
:10471000204600F093F8002383F3118805B0F0BD24
:10472000FB685A691268002AF5D01B8A013B1340C6
:10473000F1D104F15C02EAE70D3138B550F82140BF
:10474000DCB1302383F31188D4F8942413685279B0
:1047500003EB8203DB689B695D6845B10421601847
:10476000FFF770FE294604F1140001F06BFD2046AE
:10477000FFF7BAFE002383F3118838BD70470000AD
:1047800001F0CCB810B501230446282200F8243BE0
:104790000021FDF769F80023C4E9013310BD0000D2
:1047A00038B50446302383F311880025C0E903554A
:1047B000C0E90555C0E90755416001F0BFF8022383
:1047C000237085F31188284638BD000070B500EBD2
:1047D000810305465069DA600E46144618B110226E
:1047E0000021FDF741F8A06918B110220021FDF762
:1047F0003BF831462846BDE8704001F069B9000039
:10480000826802F0011282600022C0E90422C0E93D
:104810000622026201F0E8B9F0B400EB8104478996
:10482000E4680125A4698D403D4345812360002350
:10483000A2606360F0BC01F003BA0000F0B400EBCA
:1048400081040789E468012564698D403D43058141
:1048500023600023A2606360F0BC01F07DBA000019
:1048600070B50223002504460370C0E90255C0E973
:104870000455C0E906554566056280F84C5001F0C4
:10488000C3F863681B6823B129462046BDE8704021
:10489000184770BD0378052B10B504460AD080F880
:1048A00068300523037043681B680BB104219847E7
:1048B0000023A36010BD00000178052906D190F8FF
:1048C0006820436802701B6803B1184770470000F6
:1048D00070B590F84C30044613B1002380F84C308A
:1048E00004F15C02204601F0A1F963689B68B3B94A
:1048F00094F85C3013F0600535D00021204601F0BB
:1049000055FC0021204601F047FC63681B6813B189
:10491000062120469847062384F84C3070BD204677
:1049200098470028E4D0B4F86230626D9A4288BF9C
:10493000636594F95C30656D002B4FF0300380F2B5
:104940000381002D00F0F280092284F84C2083F3CB
:1049500011880021D4E914232046FFF76FFF0023BC
:1049600083F31188DAE794F85D2003F07F0343EACC
:10497000022340F20232934200F0C58021D8B3F501
:10498000807F48D00DD8012B3FD0022B00F09380C0
:10499000002BB2D104F16402226502226265A36594
:1049A000C1E7B3F5817F00F09B80B3F5407FA4D1D0
:1049B00094F85E30012BA0D1B4F8643043F00203C8
:1049C00032E0B3F5006F4DD017D8B3F5A06F31D0FA
:1049D000A3F5C063012B90D8636894F85E205E68ED
:1049E00094F85F10B4F860302046B047002884D0B7
:1049F00043682365036863651AE0B3F5106F36D02A
:104A000040F6024293427FF478AF5C4B2365022369
:104A100063650023C3E794F85E30012B7FF46DAF2C
:104A2000B4F8643023F00203C4E91455A4F86430E8
:104A3000A56578E7B4F85C30B3F5A06F0ED194F8B3
:104A40005E3084F86630204601F036F863681B68F3
:104A500013B1012120469847032323700023C4E9A2
:104A600014339CE704F1670323650123C3E723782C
:104A7000042B10D1302383F311882046FFF7C0FEAA
:104A800085F311880321636884F8675021701B68DF
:104A90000BB12046984794F85E30002BDED084F8A6
:104AA00067300423237063681B68002BD6D0022173
:104AB00020469847D2E794F860301D0603F00F01B6
:104AC00020460AD501F0A4F8012804D002287FF47A
:104AD00014AF2B4B9AE72B4B98E701F08BF8F3E7D9
:104AE00094F85E30002B7FF408AF94F8603013F038
:104AF0000F01B3D01A06204602D501F06BFBADE7DB
:104B000001F05EFBAAE794F85E30002B7FF4F5AE6F
:104B100094F8603013F00F01A0D01B06204602D598
:104B200001F044FB9AE701F037FB97E7142284F881
:104B30004C2083F311882B462A4629462046FFF74E
:104B40006BFE85F31188E9E65DB1152284F84C20EF
:104B500083F311880021D4E914232046FFF75CFE7B
:104B6000FDE60B2284F84C2083F311882B462A465D
:104B700029462046FFF762FEE3E700BFA46D000868
:104B80009C6D0008A06D000838B590F84C300446C4
:104B9000002B3ED0063BDAB20F2A34D80F2B32D886
:104BA000DFE803F037313108223231313131313130
:104BB00031313737456DB0F862309D4214D2C36849
:104BC0001B8AB5FBF3F203FB12556DB9302383F357
:104BD00011882B462A462946FFF730FE85F31188B7
:104BE0000A2384F84C300EE0142384F84C30302330
:104BF00083F3118800231A4619462046FFF70CFE5E
:104C0000002383F3118838BD836D03B198470023D7
:104C1000E7E70021204601F0C9FA0021204601F013
:104C2000BBFA63681B6813B1062120469847062328
:104C3000D7E7000010B590F84C30142B044629D06B
:104C400017D8062B05D001D81BB110BD093B022B8C
:104C5000FBD80021204601F0A9FA0021204601F0EE
:104C60009BFA63681B6813B1062120469847062308
:104C700019E0152BE9D10B2380F84C30302383F356
:104C8000118800231A461946FFF7D8FD002383F345
:104C90001188DAE7C3689B695B68002BD5D1836D07
:104CA00003B19847002384F84C30CEE70023037506
:104CB000826803691B6899689142FBD25A68036055
:104CC0004260106058607047002303758268036972
:104CD0001B6899689142FBD85A6803604260106073
:104CE0005860704708B50846302383F311880B7D60
:104CF000032B05D0042B0DD02BB983F3118808BDED
:104D00008B6900221A604FF0FF338361FFF7CEFFFB
:104D10000023F2E7D1E9003213605A60F3E70000A4
:104D2000FFF7C4BF054BD9680875186802681A6098
:104D3000536001220275D860FBF7ECBA104E0020D8
:104D400030B50C4BDD684B1C87B004460FD02B46AA
:104D5000094A684600F05EF92046FFF7E3FF009B32
:104D600013B1684600F060F9A86907B030BDFFF7DD
:104D7000D9FFF9E7104E0020E54C0008044B1A68F3
:104D8000DB6890689B68984294BF002001207047C0
:104D9000104E0020084B10B51C68D86822681A60B5
:104DA000536001222275DC60FFF78EFF014620462A
:104DB000BDE81040FBF7AEBA104E002038B5074CE6
:104DC00007490848012300252370656001F0F0FBC6
:104DD0000223237085F3118838BD00BF785000206E
:104DE000AC6D0008104E002008B572B6044B186573
:104DF00000F048FC00F0F0FC024B03221A70FEE7C2
:104E0000104E00207850002000F044B9034A516849
:104E100053685B1A9842FBD8704700BF001000E04F
:104E20008B60022308618B82084670478368A3F178
:104E3000840243F8142C026943F8442C426943F875
:104E4000402C094A43F8242CC26843F8182C02224B
:104E500003F80C2C002203F80B2C044A43F8102C06
:104E6000A3F12000704700BF2D030008104E002062
:104E700008B5FFF7DBFFBDE80840FFF751BF0000B2
:104E8000024BDB6898610F20FFF74CBF104E0020EB
:104E9000302383F31188FFF7F3BF000008B5014604
:104EA000302383F311880820FFF74AFF002383F3A0
:104EB000118808BD064BDB6839B1426818605A603A
:104EC000136043600420FFF73BBF4FF0FF30704793
:104ED000104E00200368984206D01A6802605060A5
:104EE00099611846FFF71CBF7047000038B50446AB
:104EF0000D462068844200D138BD036823605C60A1
:104F00008561FFF70DFFF4E710B503689C68A242C6
:104F10000CD85C688A600B604C60216059609968AD
:104F20008A1A9A604FF0FF33836010BD1B68121B12
:104F3000ECE700000A2938BF0A2170B504460D4687
:104F40000A26601901F02EFB01F01AFB041BA54292
:104F500003D8751C2E460446F3E70A2E04D9BDE893
:104F60007040012001F064BB70BD0000F8B5144B27
:104F70000D46D96103F1100141600A2A1969826066
:104F800038BF0A22016048601861A818144601F071
:104F9000FBFA0A2701F0F4FA431BA342064606D3A4
:104FA0007C1C281901F0FEFA27463546F2E70A2F45
:104FB00004D9BDE8F840012001F03ABBF8BD00BFBC
:104FC000104E0020F8B506460D4601F0D9FA0F4AFA
:104FD000134653F8107F9F4206D12A4601463046B9
:104FE000BDE8F840FFF7C2BFD169BB68441A2C196D
:104FF00028BF2C46A34202D92946FFF79BFF224631
:1050000031460348BDE8F840FFF77EBF104E002050
:10501000204E002010B4C0E9032300235DF8044BA8
:105020004361FFF7CFBF000010B5194C23699842C8
:105030000DD0D0E90032816813605A609A680A4442
:105040009A60002303604FF0FF33A36110BD234635
:10505000026843F8102F53600022026022699A42CE
:1050600003D1BDE8104001F097BA936881680B4402
:10507000936001F085FA2269E1699268441AA242BC
:10508000E4D91144BDE81040091AFFF753BF00BF2F
:10509000104E00202DE9F047DFF8BC8008F1100722
:1050A0002C4ED8F8105001F06BFAD8F81C40AA68C2
:1050B000031B9A423ED81444D5E900324FF0000950
:1050C000C8F81C4013605A60C5F80090D8F810303A
:1050D000B34201D101F060FA89F31188D5E90331B7
:1050E00028469847302383F311886B69002BD8D06A
:1050F00001F046FA6A69A0EB04094A4582460DD2DE
:10510000022001F095FA0022D8F81030B34208D1FD
:1051100051462846BDE8F047FFF728BF121A22443F
:10512000F2E712EB090938BF4A4629463846FFF72D
:10513000EBFEB5E7D8F81030B34208D01444211A7A
:10514000C8F81C00A960BDE8F047FFF7F3BEBDE852
:10515000F08700BF204E0020104E002038B501F02F
:105160000FFA054AD2E90845031B181945F1000159
:10517000C2E9080138BD00BF104E00200020704772
:10518000FEE70000704700004FF0FF30704700005E
:1051900002290CD0032904D00129074818BF002098
:1051A0007047032A05D8054800EBC2007047044841
:1051B00070470020704700BF986E00083823002019
:1051C0004C6E000870B59AB00546084601A9144611
:1051D00000F0C2F801A8FCF73FFB431C5B00C5E9E7
:1051E00000340022237003236370C6B201AB023483
:1051F0001046D1B28E4204F1020401D81AB070BD3B
:1052000013F8011B04F8021C04F8010C0132F0E74A
:1052100008B5302383F311880348FFF731FA0023E0
:1052200083F3118808BD00BF8050002090F85C30E7
:1052300003F01F02012A07D190F85D200B2A03D149
:105240000023C0E9143315E003F06003202B08D1DC
:10525000B0F860302BB990F85D20212A03D81F2ABE
:1052600004D8FFF7EFB9222AEBD0FAE7034A026528
:105270000722426583650120704700BF2F2300206D
:1052800007B5052917D8DFE801F019160319192009
:10529000302383F31188104A01900121FFF796FA19
:1052A00001980E4A0221FFF791FA0D48FFF7B4F971
:1052B000002383F3118803B05DF804FB302383F3EC
:1052C00011880748FFF77EF9F2E7302383F311884E
:1052D0000348FFF795F9EBE7EC6D0008106E000846
:1052E0008050002038B50C4D0C4C0D492A4604F175
:1052F0000800FFF767FF05F1CA0204F11000094931
:10530000FFF760FF05F5CA7204F118000649BDE811
:105310003840FFF757BF00BF485500203823002012
:10532000B86D0008C96D0008E26D000870B504464C
:1053300008460D46FCF790FAC6B2204601340378C1
:105340000BB9184670BD32462946FCF771FA0028A1
:10535000F3D10120F6E700002DE9F04705460C46A1
:10536000FCF77AFA2B49C6B22846FFF7DFFF08B1EF
:105370000E36F6B228492846FFF7D8FF08B1103696
:10538000F6B2632E0BD8DFF88C80DFF88C90234FB9
:10539000DFF894A02E7846B92670BDE8F08729463C
:1053A0002046BDE8F04701F03DBC252E2ED1072256
:1053B00041462846FCF73CFA70B9194B224603F1E6
:1053C000140153F8040B42F8040B8B42F9D11B78FB
:1053D000137007351534DDE7082249462846FCF7E7
:1053E00027FA98B90F4BA21C197809090232C95D36
:1053F00002F8041C13F8011B01F00F015345C95DAD
:1054000002F8031CF0D118340835C3E704F8016B27
:105410000135BFE7B86E0008E26D0008D66E0008DF
:10542000C06E0008107AFF1F1C7AFF1FBFF34F8F5A
:10543000024AD368DB03FCD4704700BF003C024043
:1054400008B5094B1B7873B9FFF7F0FF074B1A69D2
:10545000002ABFBF064A5A6002F188325A601A68B1
:1054600022F480621A6008BDA6570020003C02406A
:105470002301674508B50B4B1B7893B9FFF7D6FF9F
:10548000094B1A6942F000421A611A6842F48052CC
:105490001A601A6822F480521A601A6842F4806214
:1054A0001A6008BDA6570020003C02400728F0B54E
:1054B00016D80C4C0C4923787BB90C4D0E460823AA
:1054C0004FF0006255F8047B46F8042B013B13F0C3
:1054D000FF033A44F6D10123237051F82000F0BDB8
:1054E0000020FCE7C8570020A8570020E86E0008FD
:1054F000014B53F820007047E86E00080820704701
:10550000072810B5044601D9002010BDFFF7CEFFD3
:10551000064B53F824301844C21A0BB90120F4E7A3
:1055200012680132F0D1043BF6E700BFE86E0008D4
:10553000072810B5044621D8FFF778FFFFF780FF52
:105540000F4AF323D360C300DBB243F4007343F08C
:1055500002031361136943F480331361FFF766FF9D
:10556000FFF7A4FF074B53F8241000F031F9FFF7C1
:1055700081FF2046BDE81040FFF7C2BF002010BDEC
:10558000003C0240E86E0008F8B512F00103144632
:1055900042D185182E4A954257D82E4B1B6813F0DE
:1055A000010352D02C4DFFF74BFFF323EB60FFF7C5
:1055B0003DFF40F20127032C15D824F001046618A2
:1055C000254C401A40F20117B142236900EB010556
:1055D00024D123F001032361FFF74CFF0120F8BD24
:1055E000043C0430E7E78307E7D12B6923F44073D9
:1055F0002B612B693B432B6151F8046B0660BFF3B1
:105600004F8FFFF713FF03689E42E9D02B6923F009
:1056100001032B61FFF72EFF0020E0E723F4407326
:10562000236123693B4323610B882B80BFF34F8F9A
:10563000FFF7FCFE2D8831F8023BADB2AB42C3D080
:10564000236923F001032361E4E71846C7E700BF9D
:105650000000080800380240003C0240084908B534
:105660000B7828B11BB9FFF7EBFE01230B7008BDC7
:10567000002BFCD0BDE808400870FFF7FBBE00BF60
:10568000A65700200149024800F0A4B800FF03001B
:10569000000100200846114601F074BA084601F0E6
:1056A00087BA000038B5EFF311859DB9EFF3058493
:1056B000C4F30804302334B183F31188FFF74EFD9F
:1056C00085F3118838BD83F31188FFF747FD84F314
:1056D000118838BDBDE83840FFF740BD38B5FFF749
:1056E000E1FF114C114AC00840EA4170A0FB025E84
:1056F000C908A0FB040C1CEB050CA1FB04404FF0F7
:1057000000035B41A1FB02121CEB040C43EB000005
:1057100011EB0E0142F10002411842F100000909AB
:1057200041EA007038BD00BFCFF753E3A59BC4200A
:1057300010B50244064BD2B2904200D110BD441CB9
:1057400000B253F8200041F8040BE0B2F4E700BFC8
:10575000502800400F4B30B51C6F240407D41C6F39
:1057600044F400741C671C6F44F400441C670A4C2A
:10577000236843F4807323600244084BD2B2904202
:1057800000D130BD441C00B251F8045B43F82050F6
:10579000E0B2F4E7003802400070004050280040BA
:1057A00007B5012201A90020FFF7C2FF019803B04D
:1057B0005DF804FB13B50446FFF7F2FFA04205D0E5
:1057C000012201A900200194FFF7C4FF02B010BD1F
:1057D000704700007047000070470000074B45F21B
:1057E00055521A6003225A6040F2FF729A604CF6DA
:1057F000CC421A60024B01221A7070470030004000
:10580000D0570020034B1B781BB1034B4AF6AA224A
:105810001A607047D057002000300040034B1A68D0
:105820001AB9034AD2F874281A607047CC5700207E
:1058300000300240024B4FF08072C3F8742870476A
:105840000030024008B5FFF7E9FF024B1868C0F3CB
:10585000407008BDCC57002008B5FFF7DFFF024BB2
:105860001868C0F3007008BDCC57002070470000D6
:10587000FEE700000A4B0B480B4A90420BD30B4B40
:10588000DA1C121AC11E22F003028B4238BF00221A
:105890000021FBF7E9BF53F8041B40F8041BECE7B9
:1058A000E4700008E4580020E4580020E458002088
:1058B00070B5D0E91B439E6800224FF0FF3504EB22
:1058C00042135101D3F800090028BEBFD3F80009E4
:1058D00040F08040C3F80009D3F8000B0028BEBF99
:1058E000D3F8000B40F08040C3F8000B013263187E
:1058F0009642C3F80859C3F8085BE0D24FF0011391
:10590000C4F81C3870BD0000890141F0200101611C
:1059100003699B06FCD41220FFF778BA10B5054C3A
:105920002046FEF72FFF4FF0A043E366024B2367AC
:1059300010BD00BFD45700202C6F000870B503784D
:10594000012B054650D12A4BC46E98421BD1294BDE
:105950005A6B42F080025A635A6D42F080025A65D7
:105960005A6D5A6942F080025A615A6922F08002E7
:105970005A610E2143205B69FEF772FB1E4BE36008
:105980001E4BC4F800380023C4F8003EC023236037
:10599000EE6E4FF40413A3633369002BFCDA01238A
:1059A00033610C20FFF732FA3369DB07FCD4122095
:1059B000FFF72CFA3369002BFCDA0026A660284694
:1059C000FFF776FF6B68C4F81068DB68C4F81468EA
:1059D000C4F81C684BB90A4BA3614FF0FF336361F5
:1059E000A36843F00103A36070BD064BF4E700BF5A
:1059F000D457002000380240401400400300200229
:105A0000003C30C0083C30C0F8B5C46E05460021EB
:105A10002046FFF779FF296F00234FF001128F68AE
:105A2000C4F834384FF00066C4F81C284FF0FF303B
:105A300004EB431201339F42C2F80069C2F8006BC5
:105A4000C2F80809C2F8080BF2D20B68EA6E6B675D
:105A5000636210231361166916F01006FBD1122041
:105A6000FFF7D4F9D4F8003823F4FE63C4F8003803
:105A7000A36943F4402343F01003A3610923C4F84E
:105A80001038C4F814380A4BEB604FF0C043C4F828
:105A9000103B084BC4F8003BC4F81069C4F8003947
:105AA0006B6F03F1100243F480136A67A362F8BDC1
:105AB000086F000840800010C26E90F86610D2F89F
:105AC000003823F4FE6343EA0113C2F8003870473C
:105AD0002DE9F84300EB8103C56EDA68166806F01D
:105AE0000306731E022B05EB41130C4680460FFA8A
:105AF00081F94FEA41104FF00001C3F8101B4FF03D
:105B0000010104F1100398BFB60401FA03F391698F
:105B10008EBF334E06F1805606F5004600293AD076
:105B2000578A04F15801490137436F50D5F81C18C2
:105B30000B43C5F81C382B180021C3F81019536902
:105B40000127611EA7409BB3138A928B9B08012AF1
:105B500088BF5343D8F87420981842EA034301F1F0
:105B6000400205EB8202C8F87400214653602846C3
:105B7000FFF7CAFE08EB8900C3681B8A43EA845317
:105B8000483464011E432E51D5F81C381F43C5F814
:105B90001C78BDE8F88305EB4917D7F8001B21F402
:105BA0000041C7F8001BD5F81C1821EA0303C0E721
:105BB00004F13F0305EB83030A4A5A602846214655
:105BC000FFF7A2FE05EB4910D0F8003923F400439B
:105BD000C0F80039D5F81C3823EA0707D7E700BF1B
:105BE0000080001000040002026F12684267FFF795
:105BF0005FBE00005831C36E49015B5813F400408A
:105C000004D013F4001F0CBF0220012070470000D5
:105C10004831C36E49015B5813F4004004D013F4BB
:105C2000001F0CBF022001207047000000EB810123
:105C3000CB68196A0B6813604B68536070470000AB
:105C400000EB810330B5DD68AA691368D36019B928
:105C5000402B84BF402313606B8A1468C26E1C44BF
:105C6000013CB4FBF3F46343033323F0030302EB7F
:105C7000411043EAC44343F0C043C0F8103B2B68D3
:105C800003F00303012B09B20ED1D2F8083802EB5E
:105C9000411013F4807FD0F8003B14BF43F08053D1
:105CA00043F00053C0F8003B02EB4112D2F8003B36
:105CB00043F00443C2F8003B30BD00002DE9F04141
:105CC000244DEE6E06EB40130446D3F8087BC3F870
:105CD000087B38070AD5D6F81438190706D505EB1E
:105CE00084032146DB6828465B689847FA071FD57E
:105CF000D6F81438DB071BD505EB8403D968CCB97B
:105D00008B69488A5A68B2FBF0F600FB16228AB902
:105D10001868DA6890420DD2121AC3E900243023C1
:105D200083F311880B482146FFF78AFF84F311881B
:105D3000BDE8F081012303FA04F26B8923EA020330
:105D40006B81CB68002BF3D021460248BDE8F041BF
:105D5000184700BFD457002000EB810370B5DD6801
:105D6000C36E6C692668E6604A0156BB1A444FF45C
:105D70000020C2F810092A6802F00302012A0AB2C0
:105D80000ED1D3F8080803EB421410F4807FD4F846
:105D9000000914BF40F0805040F00050C4F80009E2
:105DA00003EB4212D2F8000940F00440C2F80009A7
:105DB000D3F83408012202FA01F10143C3F8341880
:105DC00070BD19B9402E84BF4020206020682E8A03
:105DD0008419013CB4FBF6F440EAC44040F00050A2
:105DE0001A44C6E72DE9F8433B4DEE6E06EB40132F
:105DF0000446D3F80889C3F8088918F0010F4FEA60
:105E000040171AD0D6F81038DB0716D505EB8003FB
:105E1000D9684B691868DA68904230D2121A4FF08C
:105E200000091A60C3F80490302383F311882146D7
:105E30002846FFF791FF89F3118818F0800F1CD0D6
:105E4000D6F834380126A640334216D005EB840339
:105E5000ED6ED3F80CC0DCF814200134E4B2D2F8B3
:105E600000E005EB04342F445168714515D3D5F893
:105E7000343823EA0606C5F83468BDE8F883012300
:105E800003FA04F22B8923EA02032B818B68002B8F
:105E9000D3D0214628469847CFE7BCF81000AEEB98
:105EA0000103834228BF0346D7F8180980B2B3EB39
:105EB000800FE2D89068A0F1040959F8048FC4F863
:105EC0000080A0EB09089844B8F1040FF5D81844F5
:105ED0000B4490605360C7E7D45700202DE9F74F7B
:105EE000AC4CE56E6E69AB691E4016F480586E616D
:105EF00007D02046FEF7B4FC03B0BDE8F04FFDF735
:105F000091BF002E12DAD5F8003EA2489B071EBFB3
:105F1000D5F8003E23F00303C5F8003ED5F8043859
:105F200023F00103C5F80438FEF7C6FC370505D594
:105F30009848FFF7BDFC9748FEF7ACFCB0040CD5C1
:105F4000D5F8083813F0060FEB6823F470530CBF34
:105F500043F4105343F4A053EB6031071BD563683F
:105F6000DB681BB9AB6923F00803AB612378052B11
:105F70000CD1D5F8003E87489A071EBFD5F8003EE1
:105F800023F00303C5F8003EFEF796FC6368DB6868
:105F90000BB180489847F30200F18980B70227D5FA
:105FA000D4F86C90DFF8ECB100274FF0010A09EB50
:105FB0004712D2F8003B03F44023B3F5802F11D1F0
:105FC000D2F8003B002B0DDA62890AFA07F322EAC5
:105FD0000303638104EB8703DB68DB6813B1394695
:105FE00058469847236F01379B68FFB29F42DED91E
:105FF000F00617D5E76E3A6AC2F30A1002F00F03F3
:1060000002F4F012B2F5802F00F09980B2F5402F23
:1060100008D104EB83030022DB681B6A07F5805775
:1060200090427ED13303D5F818481DD5E70302D539
:106030000020FFF743FEA50302D50120FFF73EFE37
:10604000600302D50220FFF739FE210302D50320A9
:10605000FFF734FEE20202D50420FFF72FFEA30271
:1060600002D50520FFF72AFE77037FF545AFE60747
:1060700002D50020FFF7B6FEA50702D50120FFF7E5
:10608000B1FE600702D50220FFF7ACFE210702D562
:106090000320FFF7A7FEE20602D50420FFF7A2FEC9
:1060A000A3067FF529AF0520FFF79CFE24E7E36EEA
:1060B000DFF8E0A0019300274FF00109236F9B68F0
:1060C0005FFA87FB9B453FF669AF019B03EB4B13E0
:1060D000D3F8001901F44021B1F5802F1FD1D3F876
:1060E000001900291BDAD3F8001941F09041C3F8D8
:1060F0000019D3F800190029FBDB5946E06EFFF7C1
:1061000003FC218909FA0BF321EA0303238104EB41
:106110008B03DB689B6813B159465046984701379B
:10612000CCE7910708BFD7F80080072A98BF03F88B
:10613000018B02F1010298BF4FEA182870E7023381
:1061400004EB830207F580575268D2F818C0DCF8D8
:106150000820DCE9001CA1EB0C0C002188420AD1CC
:1061600004EB830463689B699A6802449A605A68E6
:1061700002445A6056E711F0030F08BFD7F80080B9
:106180008C4588BF02F8018B01F1010188BF4FEAFD
:106190001828E3E7D4570020C36E03EB4111D1F870
:1061A000003B43F40013C1F8003B7047C36E03EBA0
:1061B0004111D1F8003943F40013C1F80039704798
:1061C000C36E03EB4111D1F8003B23F40013C1F877
:1061D000003B7047C36E03EB4111D1F8003923F443
:1061E0000013C1F80039704730B5039C01720433C5
:1061F00004FB0325C0E90653049B03630021059BB0
:10620000C160C0E90000C0E90422C0E90842C0E959
:106210000A11436330BD0000416A0022C0E9041145
:10622000C0E90A22C2606FF00101FEF75FBE000004
:10623000D0E90432934201D1C2680AB9181D7047EF
:106240000020704703691960C2680132C260C269E8
:10625000134482690361934224BF436A03610021AE
:10626000FEF738BE38B504460D46E3683BB16269B7
:10627000131D1268A3621344E362002007E0237A2F
:1062800033B929462046FEF715FE0028EDDA38BD61
:106290006FF00100FBE70000C368C269013BC36007
:1062A0004369134482694361934224BF436A436153
:1062B00000238362036B03B11847704770B5302326
:1062C000044683F31188866A3EB9FFF7CBFF054683
:1062D00018B186F31188284670BDA36AE26A13F8E4
:1062E000015BA362934202D32046FFF7D5FF002350
:1062F00083F31188EFE700002DE9F84F04460E46BE
:10630000174698464FF0300989F311880025AA46B0
:10631000D4F828B0BBF1000F09D141462046FFF761
:10632000A1FF20B18BF311882846BDE8F88FD4E98E
:106330000A12A7EB050B521A934528BF9346BBF1EF
:10634000400F1BD9334601F1400251F8040B43F8CA
:10635000040B9142F9D1A36A40334036A362403521
:10636000D4E90A239A4202D32046FFF795FF8AF325
:106370001188BD42D8D289F31188C9E730465A4600
:10638000FBF74CFAA36A5B445E44A3625D44E7E713
:1063900010B5029C0172043303FB0421C0E906130B
:1063A0000023C0E90A33039B0363049BC460C0E974
:1063B0000000C0E90422C0E90842436310BD0000A8
:1063C000026AC260426AC0E904220022C0E90A22CD
:1063D0006FF00101FEF78ABDD0E904239A4201D192
:1063E000C26822B9184650F8043B0B60704700237E
:1063F0001846FAE7C368C2690133C36043691344AE
:1064000082694361934224BF436A43610021FEF7DE
:1064100061BD000038B504460D46E3683BB1236911
:106420001A1DA262E2691344E362002007E0237AA6
:1064300033B929462046FEF73DFD0028EDDA38BD88
:106440006FF00100FBE7000003691960C268013AC0
:10645000C260C269134482690361934224BF436AE4
:10646000036100238362036B03B118477047000088
:1064700070B530230D460446114683F31188866AB1
:106480002EB9FFF7C7FF10B186F3118870BDA36A5C
:106490001D70A36AE26A01339342A36204D3E169E7
:1064A00020460439FFF7D0FF002080F31188EDE784
:1064B0002DE9F84F04460D46904699464FF0300AB4
:1064C0008AF311880026B346A76A4FB94946204689
:1064D000FFF7A0FF20B187F311883046BDE8F88FA1
:1064E000D4E90A073A1AA8EB0607974228BF1746CD
:1064F000402F1BD905F1400355F8042B40F8042B1D
:106500009D42F9D1A36A4033A3624036D4E90A23FD
:106510009A4204D3E16920460439FFF795FF8BF3D3
:1065200011884645D9D28AF31188CDE729463A46E3
:10653000FBF774F9A36A3B443D44A3623E44E5E79C
:10654000D0E904239A4217D1C3689BB1836A8BB107
:10655000043B9B1A0ED01360C368013BC360C36940
:106560001A44836902619A4224BF436A036100238B
:1065700083620123184670470023FBE700F0CCB884
:106580004FF08043586A70474FF0804300225863B1
:106590001A610222DA6070474FF080430022DA600D
:1065A000704700004FF0804358637047FEE70000DB
:1065B00070B51B4B01630025044686B058608562A8
:1065C0000E46FDF70BFC04F11003C4E904334FF051
:1065D000FF33C4E90635C4E90044A560E562FFF76E
:1065E000CFFF2B460246C4E9082304F134010D4ACB
:1065F000256580232046FEF713FC0123E0600A4A4C
:106600000375009272680192B268CDE90223074BCC
:106610006846CDE90435FEF72BFC06B070BD00BF1F
:1066200078500020386F00083D6F0008AD65000805
:10663000024AD36A1843D062704700BF104E002050
:106640004B6843608B688360CB68C3600B694361B0
:106650004B6903628B6943620B68036070470000FB
:1066600008B5234B23481A6942F0FF021A611A69E0
:1066700022F0FF021A611A691A6B42F0FF021A63D4
:106680001A6D42F0FF021A651B4A1B6D1146FFF797
:10669000D7FF02F11C0100F58060FFF7D1FF02F186
:1066A000380100F58060FFF7CBFF02F1540100F5DF
:1066B0008060FFF7C5FF02F1700100F58060FFF711
:1066C000BFFF02F18C0100F58060FFF7B9FF02F116
:1066D000A80100F58060FFF7B3FF02F1C40100F5E7
:1066E0008060FFF7ADFFBDE8084000F08FB800BF45
:1066F0000038024000000240446F000808B500F076
:106700001BFAFEF75BFBFFF789F8BDE80840FEF7D0
:10671000E9BD0000704700000F4B1A6C42F0010207
:106720001A641A6E42F001021A660C4A1B6E9368D4
:1067300043F0010393604FF0804331229A624FF09F
:10674000FF32DA6200229A615A63DA605A600122EB
:106750005A611A60704700BF00380240002004E010
:106760004FF0804208B51169D3680B40D9B2C943D4
:106770009B07116107D5302383F31188FEF744FB93
:10678000002383F3118808BD1E4B1A6962F0FF02D3
:106790001A611A69D2B21A614FF0FF301A695A6948
:1067A000586100215A6959615A691A6A62F0805227
:1067B0001A621A6A02F080521A621A6A5A6A586297
:1067C0005A6A59625A6A1A6C42F080521A641A6EF6
:1067D00042F080521A661A6E0B4A106840F48070BC
:1067E0001060186F00F44070B0F5007F1EBF4FF4CA
:1067F000803018671967536823F40073536000F002
:1068000073B900BF00380240007000403B4B3C4A67
:106810001A643C4A4FF4404111601A6842F0010288
:106820001A601A689007FCD59A6822F003029A60F1
:10683000324B9A6812F00C02FBD1196801F0F90191
:1068400019609A601A6842F480321A601A689103DB
:10685000FCD55A6F42F001025A67284B5A6F9207D3
:10686000FCD5294A5A601A6842F080721A60254A9B
:1068700053685804FCD5214B1A689101FCD5234A72
:10688000C3F884201A6842F080621A601A68120104
:10689000FCD51F4A9A600322C3F88C204FF0006297
:1068A000C3F894201B4B1A681B4B9A421B4B21D1F7
:1068B0001B4A11681B4A91421CD140F203121A6014
:1068C000164A136803F00F03032BFAD10B4B9A6897
:1068D00042F002029A609A6802F00C02082AFAD189
:1068E0005A6C42F480425A645A6E42F480425A66AC
:1068F0005B6E704740F20372E1E700BF0038024070
:1069000000040010007000400819400210300024FC
:1069100000948838002004E011640020003C02400C
:1069200000ED00E041C20F41074A08B5536903F08A
:106930000103536123B1054A13680BB150689847AE
:10694000BDE80840FDF76EBA003C014064580020E5
:10695000074A08B5536903F00203536123B1054A9E
:1069600093680BB1D0689847BDE80840FDF75ABA64
:10697000003C014064580020074A08B5536903F001
:106980000403536123B1054A13690BB15069984759
:10699000BDE80840FDF746BA003C014064580020BD
:1069A000074A08B5536903F00803536123B1054A48
:1069B00093690BB1D0699847BDE80840FDF732BA3A
:1069C000003C014064580020074A08B5536903F0B1
:1069D0001003536123B1054A136A0BB1506A9847FB
:1069E000BDE80840FDF71EBA003C01406458002095
:1069F000164B10B55C6904F478725A61A30604D58D
:106A0000134A936A0BB1D06A9847600604D5104ABE
:106A1000136B0BB1506B9847210604D50C4A936B4E
:106A20000BB1D06B9847E20504D5094A136C0BB142
:106A3000506C9847A30504D5054A936C0BB1D06CF4
:106A40009847BDE81040FDF7EDB900BF003C01409C
:106A500064580020194B10B55C6904F47C425A61FB
:106A6000620504D5164A136D0BB1506D9847230586
:106A700004D5134A936D0BB1D06D9847E00404D54B
:106A80000F4A136E0BB1506E9847A10404D50C4AFF
:106A9000936E0BB1D06E9847620404D5084A136F09
:106AA0000BB1506F9847230404D5054A936F0BB17F
:106AB000D06F9847BDE81040FDF7B4B9003C0140E5
:106AC0006458002008B50348FDF748FABDE80840BF
:106AD000FDF7A8B9A04B002008B5FFF741FEBDE8BF
:106AE0000840FDF79FB90000062108B50846FDF7EC
:106AF000B7FA06210720FDF7B3FA06210820FDF7B3
:106B0000AFFA06210920FDF7ABFA06210A20FDF7AE
:106B1000A7FA06211720FDF7A3FA06212820FDF782
:106B20009FFA07211C20FDF79BFABDE808400C21C5
:106B30002520FDF795BA000008B5FFF725FE00F007
:106B40000DF8FDF735FCFDF71BFEFDF7F3FCFFF735
:106B5000E1FDBDE80840FFF711BD00000023054A34
:106B600019460133102BC2E9001102F10802F8D1D5
:106B7000704700BF645800200B460146184600F0DD
:106B800009B80000024B0A4601461868FEF782BDAC
:106B90005823002010B5054C13462CB10A46014677
:106BA0000220AFF3008010BD2046FCE7000000008B
:106BB000024B01461868FEF771BD00BF5823002044
:106BC00010B501390244904201D1002005E003785C
:106BD00011F8014FA34201D0181B10BD0130F2E79C
:106BE0002DE9F041A3B1C91A17780144044603F115
:106BF000FF3C8C42204601D9002009E00578BD42C7
:106C000004F10104F5D10CEB0405D618A54201D11D
:106C1000BDE8F08115F8018D16F801EDF045F5D0CD
:106C2000E7E70000034611F8012B03F8012B002AC7
:106C3000F9D17047696E2E73696572726161657210
:106C40006F73706163652E507265636973696F6EEF
:106C5000506F696E7400000053544D3332463F3F0D
:106C60003F0053544D3332463430780053544D3343
:106C700032463432780053544D3332463434365829
:106C800058000000012033000010410001105A009C
:106C9000031059000710310000000000586C000874
:106CA00013040000626C0008190400006C6C0008FA
:106CB00021040000766C000840A2E4F164689106AB
:106CC0000041A3E5F265699207000000426164207B
:106CD00043414E496661636520696E6465782E00A4
:106CE0008000000000800000000080000000000024
:106CF0000000000021220008652A0008C1290008C0
:106D0000612200086D220008792400083122000861
:106D100041220008352200083D22000839220008DF
:106D20009523000845220008892D0008392D000808
:106D300055220008692300080096000000000000AA
:106D40000000000000000000000000000000000043
:106D5000714300085D43000899430008854300081B
:106D6000914300087D43000869430008554300082B
:106D7000A543000800000000B14400089D4400083D
:106D8000D9440008C5440008D1440008BD440008A7
:106D9000A944000895440008E544000800000000EC
:106DA000010000000000000063300000A86D000832
:106DB000684E00207850002053696572726120414E
:106DC00065726F7370616365005369657272612DDE
:106DD000507265636973696F6E506F696E742D428E
:106DE0004C002553455249414C250000020000004B
:106DF00000000000CD460008394700084000400070
:106E00001855002028550020020000000000000056
:106E100003000000000000007D47000800000000A3
:106E200010000000385500200000000001000000A4
:106E300000000000D4570020010102008152000828
:106E4000915100082D520008115200084300000023
:106E5000546E000809024300020100C03209040018
:106E600000010202010005240010010524010001B7
:106E7000042402020524060001070582030800FF1E
:106E800009040100020A0000000705010240000099
:106E9000070581024000000012000000A06E0008FB
:106EA00012011001020000400912415700020102C4
:106EB000030100000403090425424F415244250008
:106EC0005369657272612D507265636973696F6E83
:106ED000506F696E7400303132333435363738399B
:106EE000414243444546000000400000004000008D
:106EF000004000000040000000000100000002000F
:106F0000000002000000020000000000D14800085C
:106F1000894B0008354C0008400040004C580020C8
:106F20004C580020010000005C5800208000000048
:106F300040010000050000006D61696E0069646C2D
:106F4000650000000000002800020000AAAAAAAA0A
:106F500000000024FFFF000000000000000000000F
:106F600000A00A1500000000AAAAAA96005000007E
:106F7000FF8F00000000007788000000051000006F
:106F800000000000AA9AAAAA05000000FFFF000066
:106F900000000000000000000000000000000000F1
:106FA000AAAAAAAA00000000FFFF0000000000003B
:106FB000000000000000000000000000AAAAAAAA29
:106FC00000000000FFFF00000000000000000000C3
:106FD0000000000000000000AAAAAAAA0000000009
:106FE000FFFF0000000000000000000000000000A3
:106FF00000000000AAAAAAAA00000000FFFF0000EB
:107000000000000000000000000000000000000080
:107010000A00000000000000030000000000000063
:107020000000000000000000470400000000000015
:10703000000007000000000040420F00FE2A01008F
:10704000D2040000FF00000080500020A04B002070
:1070500000960000000008009600000000080000F4
:1070600004000000B46E00080000000000000000F2
:107070000000000000000000000000000000000010
:107080005C23002000000000000000000000000061
:1070900000000000000000000000000000000000F0
:1070A00000000000000000000000000000000000E0
:1070B00000000000000000000000000000000000D0
:1070C00000000000000000000000000000000000C0
:1070D00000000000000000000000000000000000B0
:0470E00000000000AC
:00000001FF
